:020000040800F2
:10500000F81B0020D5500008C1880008098000085E
:105010000000000000000000000000000000000090
:105020000000000000000000000000000D970008D4
:105030000000000000000000899000084998000866
:10504000E7500008E7500008E7500008E750000864
:10505000E7500008D95C0008E7500008E750000856
:1050600000000000E7500008015C0008E75000085D
:10507000E75000083185000800000000E7500008F4
:1050800000000000E75000080000000000000000E1
:10509000E750000800000000E7500008E750000853
:1050A000E7500008E7500008E750000831A1000869
:1050B000E7500008E7500008000000000000000072
:1050C0000348854600F0E8FC00480047A5B4000806
:1050D000F81B00200448804704480047FEE7FEE72D
:1050E000FEE7FEE7FEE7FEE7E5980008C15000088E
:1050F00030B50B46014600202022012409E00D4670
:10510000D5409D4205D31D469540491B25469540F7
:1051100040191546521E002DF1DC30BDF0B51FB40C
:105120000646002082B005464024019100901BE015
:10513000019922460F46304600F098FB049A059BE1
:10514000801A994110D310461946224600F07EFB82
:10515000361A8F410197224601200021009F00F05E
:1051600075FB38184D4100902046641E0028DFDC96
:10517000019B00982946324607B0F0BD03460B4319
:105180009B0703D009E008C9121F08C0042AFAD2FD
:1051900003E00B780370401C491C521EF9D2704783
:1051A000D2B201E00270401C491EFBD270470022BF
:1051B000F6E710B513460A4604461946FFF7F0FF16
:1051C000204610BD30B504460020034600E05B1CBD
:1051D000934203D2E05CCD5C401BF8D030BDF8B503
:1051E00002464A40D40F42004B0052085B089A42E4
:1051F00002D20246084611464A0023D0C30D4A0097
:10520000DDB2120EAD1A202D35DA49020126490A07
:10521000F6058A19002C00D0524220214F1B11465E
:10522000B9402A411018C20D9A4221D0002C17D043
:10523000012D08DCDA05801AD20F8019D207DBB203
:1052400000F040FBF8BDDA05801A012340001B0680
:10525000C01880185A428018CA0F1043490007E04E
:105260004908C2071143DA05801A801940088018DE
:1052700000F020FBF8BD61000122511A001BF7E786
:105280000122D2075140AAE70122D2075040A6E7E7
:1052900070B502464A40D50F40004A00ED0740086D
:1052A0005208002814D0002A12D0C40DD30D410298
:1052B0000120C0055202490A520AE41A09181218BC
:1052C0007D34914201D3641C00E04900002C01DAD6
:1052D000002070BD0023914201D3891A0343400886
:1052E00049000028F7D100290AD0914202D10121BA
:1052F000C90705E0914201D2012101E00121C94322
:10530000E005C018401900F0D5FA70BD420005D084
:105310004200120E52428A4201DB00207047C9054A
:1053200008187047F0B507460846584087B0C00FC8
:10533000049048000E46590040084908BC1A8841AC
:1053400005D2384631461E4617460B4602465800DF
:10535000400810434CD0300D039040055900400DDB
:10536000490D0590401A0290402872DA1803012175
:10537000000B09050843019004980092002805D00D
:1053800001995242002088410092019002984021E8
:105390000A1A0199009800F059FA05460C466B4626
:1053A00007CB00F074FAC0197141039A0E0D002367
:1053B000D71756401A467A40164344D0049A002A1A
:1053C0002DD0029A012A039A15DC1205C01A9141C8
:1053D00001263605001C7141D20F059ED2070093AD
:1053E000019202962A46234600F0B2FA07B0F0BDB9
:1053F00038463146FAE71605224A0F46B218C01A57
:10540000B74101210905001C4F4100187F41114699
:1054100018187941E20F10436D19644113E0E20757
:105420006D0815436408C2071443039A0126120548
:10543000C01A91413605001C7141CE074008304327
:105440004908C01851412A46234600F074FACDE7B6
:10545000FFE7049801224000C117121A00238B4174
:1054600004983146C417381AA141EEE730B401243C
:10547000E407634030BC55E730B40124E4076140E1
:1054800030BC4FE70000E0FFF0B51FB488B00B99C7
:105490000998002448400999C00F4900490809911A
:1054A000C0070B990090490049080B910999089889
:1054B000A64608431CD00B990A98084318D00998AF
:1054C00001244000420D4800410D099824050003C5
:1054D000000B204309900B980003000B20430B9016
:1054E00050181C494018002201901446104605E04F
:1054F000002001460DB0F0BD032801DA034600E0AC
:1055000003239C46C11A0AAE0AE05F0008ADED5BBA
:105510004F00F75B7D430027AA187C41491C5B1EA6
:105520006145F2DD410004AB5A522104120C0A43DA
:10553000240C401C0828DFDB01980290009970467B
:1055400001910090059B049A0799069800F000FAD3
:10555000D0E700000DFCFFFFF0B50C465C4085B0C5
:10556000E40FE40703944C000026640859009446B5
:10557000490802460296224321D062460A431ED0C1
:105580006200570D4A000E032303550D0124024605
:105590002C492405781B1B0B360B4018234326434C
:1055A000614600901C46501AB44103D30098401C39
:1055B000009002E0921800985B41002803DA002076
:1055C000014605B0F0BD00200121090507468646C9
:1055D00011E064461D46141BB54106D36546521BB7
:1055E000B341744607430C43A646CD07400849081B
:1055F000284392185B4105460D43EAD110461843F3
:1056000013D06046194650407140084306D06046AA
:10561000101AB34106D20122002306E00022012322
:10562000DB0702E00122D2435310009874460105C3
:10563000381C6141029C039D0019694100F07BF90F
:10564000BFE70000FD03000070B54B005B0803439B
:105650000BD04B005C0D002633466542B341D41796
:10566000AD1AA34102DB0020014670BD12053018BF
:10567000514170BDC217C10F504010B54018CA0744
:105680009623002100F01EF910BD10B500229623CC
:10569000114600F017F910BD0EB5C217C10F5040EA
:1056A000CA0740180021054B0293019200910A4657
:1056B0000B4600F04DF903B000BD000033040000BC
:1056C0000EB505490291002100910A460B46019151
:1056D00000F03EF903B000BD330400004100400279
:1056E0000122400AD205090E80187F2901DA002024
:1056F0007047962903DC9622511AC84070479639A4
:105700008840704770B5CD0F4A0009030123090B8B
:105710001B0519430B4BED070024520D9A4201DA89
:10572000002070BD074B34339A4203DC9A1A00F014
:105730009DF802E00449511888402C43F1D04042C2
:1057400070BD0000FF030000CDFBFFFF4A0009030E
:105750000123090B1B051943094B10B5520D9A4241
:1057600001DA002010BD064B34339A4203DC9A1A4A
:1057700000F07CF810BD03495118884010BD0000AE
:10578000FF030000CDFBFFFFC20FD207400040081F
:105790000BD0C10D0723DB01C91840020905400ADF
:1057A0001143C2084007114370470020014670476B
:1057B00010B5002904DB0124E40740428C41214656
:1057C000002B04DB1C460123DB075242A3418B4222
:1057D00000D1824210BD000010B5002904DB012475
:1057E000E40740428C412146002B04DB1C46012388
:1057F000DB075242A341994200D1904210BD000004
:10580000CB0FDB07490010B5490802460A4307D011
:105810000A0D07240903E401090B121B002A01DC0D
:10582000002010BDC900440F0C43C100E018D20590
:10583000801800F03FF810BD0122D207002800DBDD
:10584000101A002900DB511A8142704710B5202A36
:1058500004DB0146203A9140002010BD91402023F6
:105860009C1A0346E3401943904010BD10B5202A0E
:1058700004DB0846203AD040002110BD0B46D3403F
:10588000D0402024A21A91400843194610BD10B5FB
:10589000202A06DBCB170846203A1041C1170B43DC
:1058A00006E00B461341D0402024A21A9140084341
:1058B000194610BD002904DA401C490001D14008F6
:1058C0004000704770B40024050C05D1102400047A
:1058D00002D1002921D01124050E01D10002083483
:1058E000050F01D10001241D850F01D18000A41CEA
:1058F000002801DB4000641C002908D020252E1B55
:105900000D46F540A14000D001212943084301067E
:105910001B1B000ADB1D02D5002070BC7047DB0595
:10592000181880180029F8DA401C4900F5D170BC1D
:1059300040084000704710B5002B08DA0024401CD6
:10594000614192185B411A4301D14008400010BDEB
:10595000F0B51FB482B005460C0003D0084604F031
:105960009BFC02E004F098FC2030024600902146A7
:105970002846FFF76BFF049B059A04460F46184321
:105980001143084314D0184610431BD000984021FF
:105990000A1A18460599FFF769FF05460E46009A50
:1059A00005990498FFF752FF084305D0012004E051
:1059B0002046394607B0F0BD0020C11705430E430D
:1059C0002C43374300990E986305401A7905E40A81
:1059D00000220C43FD0A0A3002D500200146E9E707
:1059E0000105101969410C9C0D9D00196941FFF7D3
:1059F000A2FFDFE7FEB500231A461B1A8A4103DB2C
:105A00000020014603B0F0BD4A000D0301212D0B1B
:105A10000905520D0D43D10702D100186D41521EE8
:105A20005110FF31FF310131002704463E46384610
:105A3000009701910246012100200905FFF716FF9A
:105A4000C3197141F818324684468E464A41614670
:105A50002846611A904104D36046241A954176463F
:105A60001F46241900986D41401C00903428E1DD48
:105A7000F91930467041091BA84103D20022D243D4
:105A8000134601E00022134601980105381C7141BC
:105A9000FFF751FFB6E70000064C0125064E05E072
:105AA000E36807CC2B430C3C98471034B442F7D33F
:105AB000FFF70AFB88C30008A8C3000870B58C185C
:105AC0000578401C6B075B0F01D10378401C2A113D
:105AD00006D10278401C03E006780E70401C491C79
:105AE0005B1EF9D12B0705D40023521E0DD40B7079
:105AF000491CFAE70378401CCB1A921C03E01D787E
:105B00000D70491C5B1C521EF9D5A142D8D3002050
:105B100070BD000038B50446064805490068FFF727
:105B2000E7FA604300E0401E00900028FBD138BD3A
:105B300040420F0084010020F8B5044600688168E7
:105B40008907890F012902D10168C90722D181681B
:105B5000114A10261140012500290ED181682943E0
:105B600081600120FFF7D6FF01F028F807460CE01E
:105B700001F024F8C01B0A2807D9606D3043606526
:105B8000A06D2843A0650120F8BD20680068C043CF
:105B9000C007EDD10020F8BD170000801FB50B48ED
:105BA00000900B4801900B4802900B480390694607
:105BB0000A4804F067FF0A4A08481146083904F009
:105BC0004FFE00F06FFA002004B010BD95C1000830
:105BD00071C10008D1C10008CFC1000890010020A8
:105BE0001000002010B500231A4603E0845CE3187F
:105BF0009BB2521C8A42F9D3D84380B210BD000038
:105C000010B5034800F096FD024800F093FD10BD6A
:105C1000981700205017002030B5446C1C252C40EC
:105C20000125A540046C6560046863608368102BDF
:105C3000036803D099600068C26030BD9A60006854
:105C4000C16030BD1449012048720A4602205E320C
:105C5000507203203C3A507204200E3A50720F48A2
:105C60000D4B0078087022310870203108770C49FC
:105C70005A1C0878587149789971233318715971F1
:105C8000203318775977107551751A461E321075E2
:105C90005175107651767047E81100203E010020C2
:105CA0006001002010B503F007FD202003F0C2FDC5
:105CB000012005F051F9002003F0BCFD044804F078
:105CC000EFFF044805F09EFA002005F0D3FA10BD5E
:105CD0000001002083800000F8B503F0B9FD052025
:105CE0000121000700F056FF0025144C002800D0C9
:105CF0006560134E0221304600F04CFF002815D19C
:105D0000012020700F48808F00280ED00127BF028D
:105D100000223946304600F04AFF0A2004F010FD08
:105D200001223946304600F042FF6560012000F054
:105D300069FE022000F066FEF8BD00007001002040
:105D400000040050E80D00207047000010B508491D
:105D500000224A6107494B684C1523434B604B684E
:105D6000082423434B60C009C001026010BD00003D
:105D7000E0170020002002407FB500250C460646B3
:105D8000039500F00FFEE009029003A9019600952B
:105D9000684600F09FFD002804D000F0D7FD0020E9
:105DA00004B070BD00F0D2FD0120F9E710B500236A
:105DB00002E0C45CCC545B1C9342FAD310BD0000DB
:105DC00010B5214A00219069C305204804D54169D6
:105DD000022319434161911593699B0505D54369D8
:105DE0000124234343616302194393695B0505D58D
:105DF0004369082423434361E301194393691B0565
:105E000005D543690424234343616302194393691D
:105E10009B0405D54369102423434361630219435E
:105E200093699B0304D5446920231C4344611943AF
:105E30009369DB0305D54369402423434361A002F2
:105E40000143916110BD000000200240E0170020D6
:105E500070B5054600F0B2FE0646184C0AE0681C14
:105E600008D0002D04D000F0A9FE801BA84201D963
:105E7000032070BDA069C007F1D1A069800701D5DA
:105E80000220A061A069C00511D4A06980050ED4CC
:105E9000A06940050BD4A069000508D4A06980045E
:105EA00005D4A069800302D4A069C00303D5FFF71D
:105EB00087FF012070BD002070BD0000002002405F
:105EC000F8B51746002605460C4600F06BFD09E0C4
:105ED00029460220226800F047FD002804D1241D35
:105EE0002D1D361DBE42F3D300F030FDBE4201D25F
:105EF0000020F8BD0120F8BD10B508490246002079
:105F0000054B497905E044001C5B944203D0401CDA
:105F1000C0B28842F7D310BD8C130020700000205F
:105F200010B500F03CFE10BD10B5094801F05CF85A
:105F300080B2FFF7C5FB074A074BFFF7A5FA00221F
:105F4000064BFFF709FBFFF701FC80B210BD000014
:105F500004160020F853E3A59B843E4000408F4088
:105F600070B50024204603F027F847494748A200AF
:105F7000641CE4B28150142CF9D3464944480A7990
:105F800002754979417544490A7802764978417623
:105F90003F490520133148720A2005F023F97D207E
:105FA000400105F039F93A49002213310C2005F07F
:105FB00003FA00210C2005F011FA384801F014F81A
:105FC000344C0125223C2085AD0309E0334801F023
:105FD0000BF880B22085E18EFF392D39884206DB2F
:105FE000E18E80B28842F1D349198842EED802206E
:105FF00005F048F9002002F0DFFF294D00210F20B5
:1060000005F070F828422064F8D0206C411C38D08C
:10601000400435D58122D20100210F2005F0A1F9DD
:106020000021102005F05EF841061948490E0022B3
:10603000C73005F08DF8164DC735687A05281FD191
:1060400002221549681DFFF7BDF8002818D1114834
:10605000AE7C66710422691C3630FFF78FF8294642
:106060001331084672000D466930FFF787F86079F2
:106070002946420005484838FFF780F80320207081
:1060800070BD04F07DF90000FFFF0100EC1300205B
:106090004912002092000020600100200416002018
:1060A00000D0272410B5144C144822461032114653
:1060B000083904F0D5FB0022114BE168A068FFF716
:1060C0004BFA104A104B05F0F5FA00220F4BFFF780
:1060D000D3F900220E4BFFF7D7F9FFF791FB2060B1
:1060E00000221346E168A068FFF762FB01D0206838
:1060F00010BD0020206010BD000000209001002095
:1061000000AA8F406C45D9CC955BC83F0000F03F9A
:1061100040A5E54010B5084800F096FA0A21064867
:1061200000F032FA044800F01DF9800503D502485A
:1061300000F01AF980B210BDA8150020F8B52F4D57
:1061400000220121284600F032FDFFF7E3FFFFF7B0
:106150009CFA2B4E3146FFF79BF82A4C0122A06097
:106160001146284600F023FD2749A06800258842F3
:106170003EDB2078254F002815D02570FFF7CAFF99
:10618000FFF783FA3146FFF783F8A060FFF7FCFAC8
:1061900000223B46FFF76AF900221D4BFFF774F916
:1061A000FFF72EFB6060A068FFF7EEFA00223B4687
:1061B000FFF75CF9174A184BFFF766F906460F46DA
:1061C0006068FFF7E1FA134A144B5242FFF75CF99B
:1061D00032463B46FFF7A6F8FFF712FB1049606016
:1061E000884201DD616004E0FF21C905C84200D397
:1061F00065606068FFF772FAC0B2F8BD0004005035
:1062000000401B44480000200000604000000C409B
:1062100000E064403333333333B33040CCCCEC3F15
:106220000000C842F8B5054604464035287C0026E3
:10623000012808D001202874206881688907890F07
:1062400001290ED101E00220F8BD0168C90708D07C
:10625000606D2021084360650126002028743046C7
:10626000F8BD616DFF220132914302221143616545
:10627000C1688907890F0091C16889088900C160D8
:106280002068816892071143816000F097FC0746FF
:106290000EE000F093FCC01B0A2809D9606D0221B2
:1062A0008843102108436065002028740120F8BD50
:1062B000206880680028ECDB2068C168009A1143E0
:1062C000C160606D80088000401C6065C5E700000B
:1062D000F8B506460D464036317C01290DD0012126
:1062E000317401688A68520709D5416D2022114333
:1062F0004165002030740120F8BD0220F8BD174B25
:106300006A68D80547109A42154C8A6A2B6812D0E1
:106310005B035B0B1A438A622968490305D5A168B0
:106320000143A1600A20FFF7F5FB2868800312D51E
:10633000A06838430EE05B035B0B9A438A622968CE
:10634000490302D5A1688143A1602868800302D572
:10635000A068B843A06000203074F8BD01100000B0
:1063600000270140406D70470068006C70470000D6
:1063700070B5040006D0606D264600254036002822
:1063800002D006E0012070BDA5653574204600F0FE
:10639000D3F8606DC00603D421688868400705D52E
:1063A000606D1021084360653574EBE7606DFF2276
:1063B0000132904302221043606588688207920F81
:1063C0005B48012A02D10A68D2072BD103236268F5
:1063D0009B079A4205D05B429A4202D05B009A42E8
:1063E00009D10A69920092080A6121680A69636802
:1063F0001A430A610CE00A69920092080A618168F6
:106400000F22920491438160816862681143816028
:106410002168CA6818239A43CA602168CA68A368B9
:106420001A43CA60816801225206914381608168E3
:10643000A28E52061143816020688168C90004D48D
:10644000816801221207114381602068C168394ABE
:106450001140C1602069E168022825D00020014375
:10646000204620300278037B52035B001A4311431D
:10647000226B1143A26992031143E269D2031143D3
:106480002268D3681943D160616A0A46FF3AC23A6A
:1064900005D0A26A11432268D3681943D1604278BB
:1064A0000121012A02D00BE00420D8E7007800285F
:1064B00023D0606D202210436065A06D0843A06565
:1064C000E06B012820681FD00169C90703D001696A
:1064D00049084900016120684169C908C900416152
:1064E00020684169A26B11434161A565606D800818
:1064F0008000401C6065002070BD2068C2680123D8
:106500001B041A43C260DBE70269FF239B009A4326
:10651000026120680269236CA66C1A43636C3343E2
:106520001A430261206802690A430261D3E700004E
:10653000002701401902FEFF10B586B00446142161
:106540006846FEF734FE0E492068884216D10D4891
:10655000416B421511434163C16A01221143C1627B
:10656000C06A694610400590022000900320019007
:10657000002002900520000700F050FA06B010BD80
:106580000024014000100240F8B504464069254649
:1065900040350E4608280BD02068C068C00709D0D7
:1065A000606D202108436065002028740120F8BD3B
:1065B000082700E00C2700F001FB009011E0701CA0
:1065C0000FD0002E05D000F0F9FA0099401AB04221
:1065D00007D9606D042108436065002028740320FA
:1065E000F8BD206800683842E9D0606D0121490299
:1065F000084360652068C16809058A0F0C21002ADC
:106600001BD12022125D002A17D10268120714D56F
:10661000826853070122002B08DB43688B434360E9
:10662000606D130298431043606506E0606D20239F
:1066300018436065A06D1043A065A069002801D1D2
:10664000206801600020F8BD70B504462168002074
:106650008968490721D425464035297C01291CD069
:1066600001212974E169012904D02046FFF764FA69
:10667000002811D1616D0A4A1140FF2201321143F5
:1066800061650021A165297422681C2111602168BF
:106690008A6804231A438A6070BD022070BD00001E
:1066A000FEF1FFFF30B5014620314A790023022A6E
:1066B00004D00422C2630B71012030BD026814684B
:1066C0000E25AC431460026814686408640014600A
:1066D000446C1C22144001221546006CA540456004
:1066E0004A7118460B7130BD70B500240146203147
:1066F0004A79022A03D00421C163012418E0026808
:1067000013680E25AB431360026813685B085B00D7
:106710001360436C1C221340012215469D40036CFC
:106720005D604A7100220A71816B002900D08847A0
:10673000204670BDF0B4016C0D6801680C68466CB1
:106740001C2304221E401746B7402F420ED0670775
:106750000CD50C68A40602D40C6894430C60416C00
:1067600019408A40016C4A60016B1AE00227B74069
:1067700002462F402032002F17D0A70715D50C68EE
:10678000A40605D40C680A25AC430C6001215171A4
:10679000446C02211C40036CA1405960002111711E
:1067A000C16A002918D0F0BC08470827B7402F421B
:1067B00012D0240710D50C680E25AC430C60446C35
:1067C00001211C400B46A340046C6360C1635171FE
:1067D00000211171416BE4E7F0BC704770B5040013
:1067E0003CD01F48256814212818FEF781FC800042
:1067F00060641C482064022120462030024641711A
:1068000029681948E3680140A0686669184323694C
:1068100033431843A3691843E3691843236A1843B1
:10682000084328600121A0688903884210D00D48E0
:106830008030836A656C1C210D400F26AE40B34347
:106840008362656C63680D40816AAB400B43836271
:106850000020E06301215171107170BD012070BDF5
:10686000F8FFFDBF000002400F80FFFFF8B50446AF
:106870008C46203001790025012909D001260671B6
:1068800041790027012905D0077102252846F8BD66
:106890000220F8BD02214171E763206801684908C0
:1068A0004900016061462046FFF7B6F9206B0028D9
:1068B0002068016801D00E2205E0042291430160A6
:1068C000206801680A221143016020680168314391
:1068D0000160DBE7F8B51A4E0546307C0F4601280B
:1068E00007D0012030741748FFF7B2FA010002D038
:1068F00021E00220F8BD0020C04338606C6814E03D
:106900002046FFF723FA0F48FFF7A2FA01460E4888
:10691000426808239A434260426843159A434260A2
:10692000002901D03C6006E08034A8686A68C00194
:106930008018A042E4D8002030740846F8BD00005A
:10694000E017002050C300000020024005484168C5
:10695000022211434160416801221143416000203D
:106960007047000000200240F8B50C4C1646207C11
:106970000F46012808D0012020740948FFF768FA63
:106980000025002802D006E00220F8BD65613E60C7
:106990000348FFF75DFA2574F8BD0000E0170020FA
:1069A00050C3000011484168C9070BD0EFF31081B4
:1069B00072B60F4AC2600F4AC26081F31088416804
:1069C000C9070ED1416889070DD5EFF3108172B662
:1069D000094A0261094A026181F310884068800710
:1069E00001D50120704700207047000000200240C0
:1069F000EFCDAB8905040302BFAE9D8C16151413B1
:106A00007047000010B504494A69024202D048614B
:106A1000FFF7F6FF10BD000000040140FCB50023A5
:106A20000124A2E027462A469F403A406FD04D6895
:106A3000012D05D0022D03D0112D01D0122D16D11C
:106A400085680326AC465D00AE46AE406546B5435C
:106A5000AC46CE687546AE4065462E4386604668B5
:106A60000D79BE43ED06ED0F9D4035434560C66888
:106A70005F000325BD40AE46AE4335468E68BE403E
:106A80002E43C6604E68022E01D0122E14D1DE08AD
:106A9000B60036180196366A5D07B446EE0E0F252D
:106AA000B54000966646AE43B4460D69009EB540BB
:106AB00066462E43019D2E6206687546AE430D79EB
:106AC000AD07AD0FBD40354305604D68ED004BD5BA
:106AD000294D6E6B26436E639E08284DB6007519CE
:106AE000AC46AD689E07360F0F27B740BD4305275C
:106AF0003F07B84201D1002715E0214FB84201D12C
:106B0000012710E01F4FB84202D102270BE02BE013
:106B10001D4FB84201D1032705E01C4FB84201D1F7
:106B2000052700E00627B7402F436546AF60184DA4
:106B30002E684F689643FF0300D516432E606E689B
:106B40004F689643BF0300D516436E60AE684F682A
:106B50009643FF0200D51643AE60EE684F68964339
:106B6000BF0200D51643EE605B1C0A681546DA408A
:106B700000D057E7FCBD00000010024000000140BB
:106B80000004005000080050000C0050001C005091
:106B9000000401400069084000D0012070474269AC
:106BA00013460B401B0491430B4383617047002A3B
:106BB00001D08161704781627047000001488068A0
:106BC0007047000078010020024881680278891827
:106BD000816070477801002010B5084800240168E2
:106BE000402211430160204600F00AF8002801D03D
:106BF000012401E000F042FA204610BD00200240CE
:106C000070B504460D4D7D202978C000FEF770FA5E
:106C100001460B480068FEF76BFA00F02BFF0028D6
:106C200009D1042C07D200222146401E00F04EFA62
:106C300000206C6070BD012070BD00007801002054
:106C40008401002070477047F8B502F001FE604CE7
:106C50000120E070208AFEF718FD01467F20C00564
:106C6000FEF716FB5B4D06462968FEF7B8FA28606A
:106C70000120A16AC005814201DA084603E03046DE
:106C8000FEF702FBA062FF21C9050025C84200D320
:106C9000A562607800280BD102214F48FFF77AFFE8
:106CA00002004E494E4817D00022FFF780FFE562F0
:106CB00002214948FFF76EFF4A4E002855D0E56291
:106CC000B08AFEF7E2FC434F3968FEF7B5FD5FD2AC
:106CD0004549012008705DE00122D1034048FFF7DB
:106CE00066FF208AFEF7D1FC01467F20C005FEF733
:106CF000CFFAE16AFEF773FA3C49E0628842D7DDD9
:106D000038480127F926403000900A213046FEF726
:106D1000EFF9002903D131493148FFF701F9022188
:106D20002D48FFF737FF002801D0002701E0002F92
:106D300012D102212848FFF72DFF00280CD104F0C2
:106D400081FC00990120888005F0D8F9642003F0C7
:106D5000F7FC28492648C8600A2003F0F1FC3046B9
:106D6000761EF6B20028D0D1A2E7208AFEF78DFC6D
:106D700001467F20C005FEF78BFAE16AFEF72FFA85
:106D80001D49E06288429BDB1A491948C86097E7B1
:106D900015480570708F401EFEF76CFC3968FEF7D1
:106DA0004BFD06D82079002803D014490120087033
:106DB00001E012480570708FFEF767FC3968FEF736
:106DC0003BFD04D22079002801D004F0FFFBF8BD80
:106DD0003C010020740100200004005000800000ED
:106DE00000000050E80D0020760000200000404028
:106DF0000400FA0500ED00E00000A040860000203D
:106E0000704770B5040010D0022025462035A873C5
:106E1000204601F095FBA87B032805D0204600F012
:106E2000B9F80020A873687370BD012070BD704769
:106E3000704710B5044600680168C943C90708D106
:106E40008168C943C90704D1012141602046FFF789
:106E5000FBFE20680168C943890708D48168C943DB
:106E6000890704D4022141602046FFF7EBFE206829
:106E70000168C943490708D48168C943490704D454
:106E800004214160204600F0F7F820680168C943FA
:106E9000090708D48168C943090704D4082141605F
:106EA0002046FFF7ADFF20680168C943C90608D432
:106EB0008168C943C90604D4102141602046FFF708
:106EC000C2FE20680168C943890608D48168C943A5
:106ED000890604D4202141602046FFF7A9FF2068DD
:106EE0000168C943490608D48168C943490604D4E6
:106EF000402141602046FFF79AFF10BDF8B504001D
:106F000005D025462035A87B002802D006E00120C8
:106F1000F8BD00206873204600F04EF80220A873E8
:106F20002068C26884466368012B01D10620824331
:106F300016486169814202D0072040038243002B3A
:106F400001D1D82082431248A66802401846304337
:106F5000676A266A3E433043A66A30431043002BDB
:106F600002D0012B04D005E02369E2691A4300E056
:106F7000E2681043054A914202D0A26911430843D6
:106F80006146C8600120A8730020F8BDFFFF000023
:106F9000F8F119FF10B500680549884207D1054886
:106FA000816B4900490881630D2000F073F810BD22
:106FB000007C00400010024010B50068084988427B
:106FC0000CD10848816BC204114381630022012166
:106FD0000D2000F07BF80D2000F06CF810BD0000D3
:106FE000007C0040001002400068C069704700004B
:106FF000F8B504460220254620351746A8731D48DB
:107000000268C3041A4302602068C2689B121A43D4
:10701000C2602068026901263243026122681020A2
:107020005060206881611021204601F0F9FA0328A0
:107030001FD0216808204860206847610821204649
:1070400001F0EEFA032814D0204601F079FAA87B6B
:1070500003280ED02068816831438160206801696F
:107060003143016120680169042211430161AE735B
:107070000020F8BD00040140704700000448416B47
:10708000012211434163816B020411438163704704
:1070900000100240002809DBC106C90E012088400B
:1070A00003490860BFF34F8FBFF36F8F7047000035
:1070B00080E100E0002805DBC106C90E0120884000
:1070C000014908607047000000E100E010B503F0DE
:1070D00035F910BD02494A6882434A607047000092
:1070E000007000400248016882151143016070473A
:1070F0000070004002494A6802434A60704700003D
:1071000000700040054801680222114301600448F4
:10711000016904221143016130BF704700700040D3
:1071200000ED00E0F0B5154A1368154D54152D6AB1
:107130002340ED07ED0F002B04D0002D02D0166880
:10714000A64316601668B608B600064316600D48DA
:10715000076904263743076101290DD040BF20BFCE
:1071600020BF0169B1430161002B04D0002D02D082
:10717000106820431060F0BD30BFF2E7007000409F
:107180000000014000ED00E0F8B50446007800275B
:10719000534D800671D5524E403EB06BC00004D4B2
:1071A000B06BA9050843B06301274E480168C905C3
:1071B00011D40168821511430160FFF7FFFC0090B4
:1071C00005E0FFF7FBFC0099401A642837D84548D2
:1071D0000068C005F5D532680321090560680A40DA
:1071E0000140914208D08103890F032904D13168FD
:1071F000890301D50120F8BD2A69032109040A4049
:1072000022D0084090421FD0207880061CD52869E3
:107210002A6988430121C9040A432A612A698A43E9
:107220002A612861C0050FD5FFF7C8FC009008E06F
:10723000FFF7C4FC0099411A2B48814201D9032071
:10724000F8BD28698005F3D561688803800F03289D
:1072500005D132680005824301400A433260286943
:10726000032261681204114008432861002F04D0F2
:10727000B16B012000078143B1632078C00705D0BE
:10728000E868A168800880000843E86020788007EB
:1072900005D5E8680C218843E1680843E860207858
:1072A000400706D5E868032189028843216908431D
:1072B000E8602078000706D5E868032109038843C1
:1072C00061690843E8602078000606D5E868032174
:1072D00089048843A1690843E8600020F8BD0000E4
:1072E000401002400070004088130000F8B50E46C0
:1072F000050038D05E480068C007C00FB04214D205
:107300005B4C20684008400030432060FFF756FC8B
:10731000074605E0FFF752FCC11B564881427AD868
:107320002068C007C00FB042F4D12878524C8007C3
:1073300005D5E068F0218843A9680843E060287813
:10734000C00752D06868022806D0032807D02168F9
:1073500001280AD0890504E02168890301E0216839
:107360008901002903DB0120F8BD4907F9E7E1683D
:10737000890889000143E160FFF720FC074668683F
:1073800002280AD0032814D001281ED029E0FFF7D4
:1073900015FCC11B374881423DD8E0680007800FCB
:1073A0000228F4D121E0FFF709FCC11B31488142DA
:1073B00031D8E0680007800F0328F4D115E0FFF70B
:1073C000FDFBC11B2B48814225D8E0680007800FD8
:1073D0000128F4D109E0FFF7F1FBC11B25488142E8
:1073E00019D8E0680007800FF5D121480168C90766
:1073F000C90FB14217D901684908490031430160FA
:10740000FFF7DCFB074608E005E0FFF7D7FBC11BF1
:107410001848814201D90320F8BD15480068C0070B
:10742000C00FB042F1D12878400706D5E0680721A7
:1074300009028843E9680843E0602878000707D517
:10744000E0680721C90288432969C9000843E06050
:1074500000F03AF8E168094A0906090F515CC84092
:107460000749086007480068FFF7CAFBF8BD00003D
:10747000002002408813000000100240D6C200081D
:10748000840100207C010020044805490068C96887
:10749000044A4905490F515CC840704784010020E7
:1074A00000100240EFC20008044805490068C9689E
:1074B000044A8904490F515CC84070478401002088
:1074C00000100240EFC2000870B51A4AD3681A498A
:1074D0000C2018408D0004280CD04E00082810D035
:1074E0000C2810D050680004410F0120C003491C33
:1074F000884070BD1068C00601D5084670BD28469A
:1075000070BD304670BD98020C4C000F205C1B0211
:107510009C0FD368641CDB0301D5314603E012687D
:10752000D20600D4294602F0CEFE22460023FDF703
:10753000F5FD70BD0010024000093D00E6C20008E4
:10754000FEB505007ED0FE4CE7680C20E6680740DB
:107550000120000406402878C00747D0082F05D036
:107560000C2F0AD101200004864206D12068800336
:107570003CD568680028E5D038E00120696800043F
:10758000814203D121680143216011E005230122DA
:107590001B0492049942216802D111432160F1E752
:1075A0008143216021680140009120689043206060
:1075B000686800280DD0FFF701FB009005E0FFF799
:1075C000FDFA0099401A64287BD820688003F6D51C
:1075D0000CE0FFF7F3FA009005E0FFF7EFFA0099EF
:1075E000401A6428F0D820688003F6D428788007F1
:1075F00056D50923E868042F0DD00C2F01D1002E99
:1076000009D000283CD02168994301432160FFF74D
:10761000D5FA064628E02168490701D5002891D00F
:1076200061681F22120291432A69120211436160AC
:107630002168994301432160FFF746FFE16809068D
:107640000A0F00E08BE1BF49895CC840BE49086071
:10765000BE480068FFF7D4FA002873D120E0FFF796
:10766000ADFA801B0228AFD820684007F7D56068C4
:107670001F210902884329690902084360600FE05D
:107680002068400840002060FFF798FA064604E0B2
:10769000FFF794FA801B022896D820684007F7D499
:1076A0002878C00660D5002F0CD0A86900284AD0E1
:1076B0002068FF21013108432060FFF77FFA06466A
:1076C0002EE0C1E02068800502D5A8690028A6D078
:1076D0006068072149038843296A0843606060683D
:1076E000297F0002000A090608436060286A410BEE
:1076F0000120C003491C8840E16809060A0F91492E
:10770000895CC8409049086090480068FFF778FAA3
:10771000002817D128E0FFF751FA801B0228A2D8D1
:1077200020688005F7D56068072149038843296AE6
:10773000084360606068297F0002000A0906084368
:10774000606011E0E2E02168FF20013081432160A8
:10775000FFF734FA064604E0FFF730FA801B0228F0
:1077600072D820688005F7D42878794E000724D590
:1077700068690028306910D0012108433061FFF7A3
:107780001DFA009005E0FFF719FA0099401A022847
:107790005AD830698007F6D50FE0400840003061C4
:1077A000FFF70CFA009005E0FFF708FA0099401A7D
:1077B000022849D830698007F6D42878400766D572
:1077C00000200290A06BC00006D4A06B0121090725
:1077D0000843A063012002905E480168C90511D4E6
:1077E0000168821511430160FFF7E8F9009005E098
:1077F000FFF7E4F90099401A642825D85548006835
:10780000C005F5D5FF20AA680130824203D1316955
:107810000143316111E001218902002A07D00523CB
:107820001B029A4203D132690A433261EFE732699F
:1078300082433261306988433061A868002810D0E3
:10784000FFF7BCF9009008E05FE0FFF7B7F90146E9
:107850000098091A4048814257D830698005F4D50C
:107860000DE0FFF7ABF9009006E0FFF7A7F90099EC
:10787000411A3948814248D830698005F5D40298C8
:10788000002804D0A06B012109078843A063686A1F
:10789000002866D00C2F3ED001263606022820682C
:1078A00005D0B0432060FFF789F905462FE0B043CB
:1078B0002060FFF783F9074604E0FFF77FF9C01B5C
:1078C000022822D820688001F7D4E96AA86AE26811
:1078D0000843296BFD231B049A4311430843E060CE
:1078E000206830432060FFF769F9054604E0FFF7A0
:1078F00065F9401B022808D820688001F7D530E0E0
:10790000FFF75CF9401B022801D90320FEBD206867
:107910008001F5D425E00128F8D0E06801210904B0
:10792000AA6A014091421AD10F218904EA6A0140F2
:10793000914214D1032189050840296B88420DE04A
:1079400000100240D6C20008840100207C01002003
:1079500040100240007000408813000001D0012058
:10796000FEBD0020FEBDF8B504000ED0FF27606A02
:107970000537002500280AD0256165612646403676
:10798000A562707C002807D00AE00120F8BD60687D
:10799000B842F3D0E561F1E73574204600F03EF8D7
:1079A000022171742068026840239A4302602123F7
:1079B000A26860689B021A4038401043E3688A025C
:1079C0001340184323690B40217D1843C907C90F91
:1079D0000843A169931019400843E169382319400D
:1079E0000843216A802319400843A16A9300194083
:1079F000084321680860A0690421000C0840616AFE
:107A0000102319400843216848602068C1699143E8
:107A1000C1616565012070740020F8BD10B586B0A5
:107A2000044614216846FDF7C2FB104920688842CD
:107A300019D10F48416B821411434163C16A01227D
:107A40001143C162C06A002110400590E0200090FF
:107A500002200190032003900291049105206946C1
:107A60000007FEF7DBFF06B010BD0000003001404C
:107A700000100240094910B5401E884201D901207A
:107A800010BD074C60610321081F02F057FC002065
:107A9000A06107202061002010BD0000FFFFFF0053
:107AA00000E000E070B505462C4602202034002995
:107AB00008D004290BD008290ED0627F012A10D0EB
:107AC000012070BDA27E012AFAD1A0760AE0E27EF2
:107AD000012AF5D1E07605E0227F012AF0D1207756
:107AE00000E060770122286801F028FF0122286861
:107AF00092070121904205D0074A904202D0074ADE
:107B0000904204D182685207520F062A02D00268BE
:107B10000A430260002070BD0008014000140140CB
:107B200070B504460D460068002201F007FF20688A
:107B3000016A0C4A114203D10168490849000160F9
:107B400001202034002D06D0042D06D0082D06D0AB
:107B50006077002070BDA076FBE7E076F9E720773C
:107B6000F7E70000111100007047704770470000F0
:107B7000F8B502680446D06911689668814B0546DD
:107B80001D402023002D6CD0F7077F4DFF0FBC4612
:107B90000D402F4379D02546C7078035002F06D0EA
:107BA000CF0504D5012717622A683A432A60820765
:107BB00008D5F20706D0276802223A622A6804270D
:107BC0003A432A60420708D5F20706D02668042205
:107BD00032622A68022632432A6002070AD50A4620
:107BE0001A406646324305D02668082232622E6863
:107BF00016432E60020508D54A0106D501222668E3
:107C0000D20232622A681A432A602A68002A30D0D7
:107C1000800606D5880604D5616E002901D020466D
:107C20008847286821688968490602D428210842C3
:107C300025D0204602F093F820688168490619D5BE
:107C4000826840218A438260206F002812D04F4909
:107C50008163206FFEF748FD00280AD0206F816BFA
:107C600006E0850611D58D060FD5616E77E02046BA
:107C70008847F8BD2046FFF779FFF8BD05E02046AC
:107C8000FFF774FF00202860F7E7256E012D56D11D
:107C9000C50654D5CD0652D51026166220688168D7
:107CA00025464906403500292ADA226F11684968BD
:107CB0000904090CE1D02F8B8F42DED9698311684A
:107CC0000968890617D40168320191430160206870
:107CD0008168490849008160206881684022914399
:107CE0008160E3670020206620680168B14301607D
:107CF000206FFEF7D7FC288B698B401A81B21AE0FF
:107D0000298B6A8B891A6A8B89B2002AB5D000291F
:107D1000B3D00268FF252135AA430260206882683B
:107D2000520852008260E367002020666066206887
:107D30000268B24302602046FFF716FF9DE7C502C6
:107D400008D5750206D50120000510622046FFF710
:107D50000CFF92E7050605D50D0603D5A16E002997
:107D600085D18AE7400688D5480686D51168204621
:107D70004024A143116083670021816600F043F92C
:107D80007BE700000F08000020010004859C00082C
:107D900010B5040003D0A06F002802D007E0012036
:107DA00010BD002174200155204600F027F8242042
:107DB000A06720680168490849000160204602F078
:107DC00021F80128ECD0606A002802D0204601F09A
:107DD00043FE206841680922D20291434160206835
:107DE00081682A2291438160206801680122114341
:107DF0000160204601F096FE10BD0000F0B587B08E
:107E0000064614216846FDF7D2F92C4930688842AD
:107E100051D12B48416B0122920311434163C16A46
:107E200001221143C162C06A002510400590032061
:107E3000400200900220032701A9A1C10420049060
:107E4000052069460007FEF7E9FD1F4C1D48A560A7
:107E5000E56081C48027E560A7602020256160611E
:107E60000002A0611848083CFEF7B8FC002801D0C9
:107E7000FDF76AFF3467A662144C12482146143895
:107E800020600320606010200831A1C16561A561F8
:107E9000E56120462562FEF7A1FC002801D0FDF730
:107EA00053FFF466002201211B20A662FFF70EF9A2
:107EB0001B20FFF7FFF807B0F0BD000000380140BD
:107EC0000010024030000240501700209817002098
:107ED00070B5C36F202B27D100290BD0002A09D001
:107EE000012483682403A34206D10369002B03D134
:107EF000CB0701D0012070BD034660331C7D012CEF
:107F000012D001241C7500230366084C0368A342A9
:107F100007D05C68240204D51C680125AD062C43FB
:107F20001C6002F06FF870BD022070BD0048004078
:107F300070477047FFB50446806F83B017460D4603
:107F400020285ED1002D0AD0002F08D0A168C001E2
:107F5000814207D12069002804D1E80702D001201E
:107F600007B0F0BD204660300090007D012848D069
:107F70000098012101750020802108512120A0676F
:107F8000FEF71CFE2646403601903782778201209C
:107F9000A1680003814202D12069002805D02F4644
:107FA000002500990020087511E00027F9E700225C
:107FB0008021204602F06CF8002815D1002F15D042
:107FC0002168387888627F1C708A401E7082708AAF
:107FD000019B002806980090E9D10022402120460C
:107FE00002F056F8002808D00320B9E72888216855
:107FF000C005C00D8862AD1CE6E72020A067002008
:10800000AEE70220ACE77047034D044C04A002F039
:1080100039F9E560FAE700000400FA0500ED00E038
:10802000486172644661756C745F48616E646C652A
:10803000722E0D0A0000000070B586B0142168464B
:10804000FDF7B5F801240B480C4EC4800A48A50280
:108050004483224629463046FEF7A9FD00210291BD
:1080600003910095019469463046FEF7D7FC06B0AF
:1080700070BD0000280E00203C01002000040050CC
:1080800010B505242407002204212046FEF78FFDA9
:10809000002208212046FEF78AFD0A2002F057FB45
:1080A000012204212046FEF782FD0A2002F04FFB48
:1080B000002204212046FEF77AFD10BD10B50524EC
:1080C0002407002204212046FEF771FD0122082129
:1080D0002046FEF76CFD0A2002F039FB0122042144
:1080E0002046FEF764FD0A2002F031FB0022042145
:1080F0002046FEF75CFD10BDF8B5002405260746B6
:1081000025463607002204213046FEF750FD0A209E
:1081100002F01DFB012204213046FEF748FD6006F7
:10812000040E08213046FEF735FD002801D0641CFE
:10813000E4B2052002F00BFB6D1CEDB2082DE1D37B
:10814000002F03D0FFF79CFF2046F8BDFFF7B6FFD6
:10815000FAE770B5052605463607002204213046A9
:10816000FEF725FD0024E80901D0012200E00022ED
:1081700008213046FEF71BFD6806050E0A2002F0B6
:10818000E6FA012204213046FEF711FD0A2002F032
:10819000DEFA002204213046FEF709FD0A2002F033
:1081A000D6FA641CE4B2082CDDD370BD10B50524EA
:1081B0002407012208212046FEF7F9FC01220421B0
:1081C0002046FEF7F4FC002208212046FEF7EFFCD3
:1081D0000A2002F0BCFA002204212046FEF7E7FC48
:1081E00010BD10B505242407002204212046FEF707
:1081F000DEFC002208212046FEF7D9FC0A2002F00E
:10820000A6FA012204212046FEF7D1FC0122082112
:108210002046FEF7CCFC0A2002F099FA10BD70B59A
:1082200005252D070024012208212846FEF7BFFC62
:10823000062002F08CFA012204212846FEF7B7FC42
:10824000062002F084FA07E0641CE4B2FA2C03D999
:10825000FFF7C7FF012070BD08212846FEF79AFCF2
:108260000028F1D1002204212846FEF7A0FC0020BE
:1082700070BD0000F8B501F087FC01F0B7FC5B4869
:108280000068C069FDF750FE594C5A49A082898F99
:10829000594E0025002931D0A26A730357499A42EA
:1082A00002DB02220A7000E00D700A7801218902C7
:1082B000002A05D0012A0ED0022A10D0032A1DD18F
:1082C000608B01282ED0022818D148480821403858
:1082D000FFF726FC12E0FF22F5329042F0D2608BCD
:1082E00001281DD0022804D008E03046FEF75FFCCC
:1082F00004E03E4808214038FFF7D4FBFDF71EFF9D
:1083000020700121C9023046FEF744FC0127FF031B
:1083100000282DD03A480560A079002804D007E055
:108320000022E2E70122E0E70120A07101F012FF44
:1083300080213046FEF72EFC002806D000220821BE
:108340003046FEF734FC012205E0012208213046C8
:10835000FEF72DFC0022052039460007FEF727FC1A
:10836000244C284E4034A08C274F012803D01CE019
:10837000A5710022EAE725486946088072B6802187
:108380002348FDF7F9FC002804D002226946204862
:10839000FDF796FD62B61FA001F074FFA58403F0FF
:1083A000ADFE642002F0CCF9FE60608C012808D19B
:1083B00010486584058003F0A1FE642002F0C0F936
:1083C000FE60208C012806D1258403F097FE6420EE
:1083D00002F0B6F9FE600748124A0188914202D1C4
:1083E000C088002800D1FE60F8BD0000CC16002037
:1083F0003C010020E80D0020000400508400002013
:10840000740100200400FA0500ED00E0AAAA0000B3
:10841000384A0008BDF8C8EBC9FDBCB6C4A3CABD44
:108420000D0A0000AA55000038B55721202000F0A1
:108430007AF80321212000F076F84021222000F074
:1084400072F80821232000F06EF8AA21302000F0F5
:108450006AF81048018F142901D8002901D101219F
:1084600001870C4C40346188142901D8002901D1BE
:1084700002216180008FC1B2322000F054F8A1784F
:10848000332000F050F8684600F006F80A2002F0A9
:108490005EF938BDE80D002010B501460F2000F050
:1084A00021F8002800D0012010BD10B50446FFF7C8
:1084B0007DFE3220FFF74DFEFFF7B1FEE0B2FFF781
:1084C00048FEFFF7ACFEFFF771FE3320FFF741FED9
:1084D000FFF7A5FE0020FFF70FFE0446FFF781FE21
:1084E000204610BD10B50C46FFF7DFFF20700120BD
:1084F00010BD70B50D460446FFF758FE3220FFF759
:1085000028FEFFF78CFEE0B2FFF723FEFFF787FEA1
:108510002846FFF71EFEFFF782FEFFF762FE0A20E5
:1085200002F015F970BD10B5FFF7E3FF012010BD93
:1085300010B50248FEF77DFC10BD000004160020B7
:10854000FEB50446002772B6334A01688B1804D181
:108550003248C76803208004074088680190C868D3
:10856000009048698E69002B08D12C4940398B6AEC
:10857000CD042B438B628B6AAB438B620146314344
:108580003CD025492368CB4205D12449CA6803233E
:108590009B049A43CA6025462035002810D02168E4
:1085A0000A6901231A430A612168486108212046AB
:1085B00000F036F8032800D1A8732168082048602D
:1085C000002E10D02068016901221143016120684A
:1085D00086611021204600F023F8032800D1A873FB
:1085E0002168102048600C482168C14206D10B4820
:1085F000C1680322920491433943C1602068016934
:108600004908490001612168019888602168009843
:10861000C86062B6FEBD00000084FFBF401002408B
:1086200070B506460B480D46002409490068FCF762
:108630005FFD7D21C90048433168401E00D10324FD
:108640000B682A469A4301D00028F6D1204670BD17
:10865000204E0000840100201CB500211648009126
:10866000144A01910260C1631205426081600722D1
:108670008263012202610246C16020321170FF2331
:108680005170C233436281621173016381610422BC
:1086900041634261C161FDF76BFE084800908013A1
:1086A000019069460448FDF713FE00210248FDF7DA
:1086B000B9FD1CBD00240140A815002002000004E3
:1086C00008B50848016B012211430163006B0121C9
:1086D0001040009000220A20FEF7F8FC0A20FEF766
:1086E000E9FC08BD00100240F0B587B014216846CF
:1086F000FCF75DFD4748C26A04210A43C262C26AB0
:108700000A400592C16A80263143C162C16A314084
:108710000591C16A01242143C162C16A21400591CA
:10872000C16A02252943C162C06A224628400590D9
:1087300005201C210007FEF73AFA01223649374886
:10874000FEF735FA002236493448FEF730FA912117
:108750000520002209020007FEF729FA314801909E
:10876000002705206946029700940007FEF756F996
:108770000C20009011200190032003900520029707
:1087800069460007FEF74AF910206A46039591C230
:10879000052069460007FEF741F911200190029774
:1087A0006946039700941D48FEF738F91E4801906A
:1087B0006946009502941948FEF730F9E0020090EE
:1087C0006946019702951548FEF728F9174869464A
:1087D00091C1694611480397FEF720F991200002E4
:1087E000694691C10520694600070397FEF716F90F
:1087F00069460A48019700960294FEF70FF9002295
:1088000001210520FEF762FC0520FEF753FC07B0AE
:10881000F0BD000000100240010200000004005002
:108820000830000000001110000021100832000084
:1088300010B50F4C0D482060FF200530606000200F
:10884000A060E06020616061E06101212062490276
:108850006062A161A0620720E0622046FFF783F812
:108860002068016840221143016010BD00300140C2
:108870003416002000B585B014216846FCF797FC3B
:108880000E480D490160E1214902416000218160EB
:10889000C160016181610C22C161426101623021CC
:1088A00041620121090381634900C163FFF770FA46
:1088B00001F04AFC05B000BD00380140CC16002094
:1088C00070470000F0B589B00A2002F08BFC7D20D3
:1088D000400102F0A1FCFF4C0025A570FE48206677
:1088E000607C0C2801D30B20607460790A2801D9C0
:1088F0000A206071F948E570F94E00783071F94945
:10890000A079097840000843A17D89000843F071EF
:10891000E06BF070010A3172401CE0636079B07462
:1089200042003046F0491330FCF728FC6079EE49EC
:1089300082004000801960311330121DFCF71EFCCC
:1089400060790621420048438019E8491730921C9B
:10895000FCF714FC2E20205E002803D0E449098A8D
:108960000818E0856079DB49C000223182190B7B51
:1089700053764B7B937606227272DE4A1D30127854
:10898000B272A28C3273D64A0B79133A13754979B5
:1089900051750022D24902F00FFD60790021C0001C
:1089A0001D3002F01BFDD448FEF71EFB0127208579
:1089B000BF0309E0D048FEF717FB80B22085E18EA7
:1089C000FF392D39884206DBE18E80B28842F1D32F
:1089D000C9198842EED8022002F054FCC048012692
:1089E000C571A574A5732674E573C348FEF7FCFA38
:1089F00060850746E5706079FCF762FEBF4AC04BB0
:108A0000FCF742FD01F038FE0022BE4BFCF78AFC69
:108A1000FCF79CFE0006C10CC81980B2F103A085CA
:108A2000884201D3401AA085B748E0642079401CF1
:108A30002071B148FEF7D8FA2085AB48A54F6438BD
:108A400040370690B1E1AC48FEF7CEFA20850BE046
:108A5000A948FEF7C9FA80B22085A18D884203D3C8
:108A6000AA4A8918884207D300210F2002F03AFB56
:108A7000A74920640842EBD0206C411C1FD0400461
:108A80007ED58122D20100210F2002F06AFC002154
:108A9000102002F027FB41069348490E00227C3843
:108AA000E16502F055FB002002F0B6FB002002F069
:108AB00068FB8D487C38417A0729C3D101E001F079
:108AC0005FFC02229349401DFCF77CFB0028B9D1D2
:108AD00002F0D5FCE167A06702F0BEFC7D4B80335D
:108AE00003C3E0788049401CE07083390B7A684604
:108AF0000370497A417000880390E18C88427DD1EF
:108B0000774985488C31C98E0180754971488C310F
:108B1000098F41847848FEF767FA208502F0F4F95E
:108B20006C48FF2280300168406852040023891895
:108B300058410206080A10434108490000900A0EF5
:108B4000080264498031CA6088606548E36F0A3072
:108B5000A26F02F069FC60798100614808185D49E4
:108B6000163080310CC902F05FFC5A488030C3686F
:108B700082685B48123002F057FC0821584800E038
:108B800006E14172B430C07C0009607514D05648CB
:108B9000022260497738FCF715FB00280CD15048B9
:108BA000A674C671E06D50491638C2B26639C81D48
:108BB000E274FB30FCF7E2FA607900228000484959
:108BC0001C3002F0F9FB6079002180001C3002F0BB
:108BD00005FC009802F0FFFA012002F053FB20731D
:108BE00002214E48FDF7D6FF00281DD000213D4848
:108BF00001703B498C31488E049000E05AE0388186
:108C0000888E78818446A06CFF310531E06408606D
:108C1000DC392065C97C0907090F032900D02175BB
:108C2000E16D1C2902D015E00121E0E72C49294A19
:108C30008C31C98F1186069B2C4A1B881380884271
:108C400007DD002805DD002903D0207E401C2076AA
:108C500000E025762571A6730498B8816046F881F6
:108C6000E673608C2E49FF30C33080B26084884246
:108C70000CD949424018608427487D220188D200DF
:108C8000491C89B20180914200D3058022487D2190
:108C90000088C9004843618C4018606500F074FD8D
:108CA000207B002805D100210F2002F01BFA0006CE
:108CB000F9D583E0FDF720F90B4A032190321154D6
:108CC00007498C314A8E3A81898E7981E26D1C2A5E
:108CD0002ED127E0700000203F420F003C01002011
:108CE0005C120020700100208C130020C8140020AA
:108CF000280E00204C01002004160020B81E85EB31
:108D000051B8CE3F00000840A0860100983A00000C
:108D100000D02724600100206C01002000040050D6
:108D2000E7030000614B4200D318069A12885A806C
:108D300080005F4B5E4AD43B02905D4982189B8F56
:108D4000138030314118A26C4A605A4940185A4980
:108D500016300CC902F068FB216EA06C884207DA5D
:108D6000534A02995158012902D12066039905916D
:108D70004F49029A8958814217DD012915DD2146A4
:108D8000002812DD0398C8840220087065730CE087
:108D90004A4A00210F2002F0E4FA6079E178401C91
:108DA000814202D0002002F0ECF9208DA18D884292
:108DB00000D248E6424A89188842FAD8A07B0128A6
:108DC00001D00220A07302F09FF83C4A00210F203E
:108DD00002F0C7FA2079002817D03A4909888A009A
:108DE0008A18824200D22570002000F0E5F8A07CAD
:108DF000002839D02E496C310B78A3724878607204
:108E00008A782272022B17D02EE0E16C226E323962
:108E100020468A420EDAC1792A4A491CC9B2C17178
:108E2000128852008A42E2D20599C184022101705F
:108E30006573DCE7E571DAE710280CD0C82813D297
:108E4000214BC91C1818FCF799F903F057F9642055
:108E500001F076FC33E61D4D28684000000E03D17A
:108E6000C878FCF712FC286000202378627B6579C3
:108E70000FE00F4E4100303E775A1836765AB7420F
:108E800005D00B4F022300220126483F7E52401C92
:108E9000C0B2A842EDD323706273084A0021803229
:108EA0000F2002F05EFA09B0F0BD0000C8140020E7
:108EB000BC1300205C120020F000002000D027240A
:108EC000983A00004C010020E80D002064010020C9
:108ED000F8B52E4C0546E06E2D4A281A411E206733
:108EE000914215D21A21615E081AFCF7D5FB294A76
:108EF000294BFCF7C9FA064632200F46205EFCF7E4
:108F0000CBFB32463B46FCF70DFAFCF7FBFB6086D9
:108F1000002060761D481C23C35E828C1F48008899
:108F200084461F4806881DE06046484380181D4F50
:108F300080B23880302778436427643078431A4FF2
:108F40006066C01985420BD2C8B218493222088027
:108F5000606EA25E411BC9188918A166E066F8BD63
:108F6000491C6176617EB142DED330204243104815
:108F70006421101848430F494118E16660663221A8
:108F8000401B615EC0184018A066F8BD700000204C
:108F9000CF0700009A9999999999B93F5A010020F1
:108FA0004C0100206E01002078ECFFFF58010020EA
:108FB00074270000C0BDF0FFFEB5294D2988491C6B
:108FC0008FB228492F800E88FCF766FB264A274B74
:108FD000FCF75AFA0191009025483146FCF788F8D1
:108FE000244C218F4218B74206D300202880224803
:108FF000019E1018009D02E01046019E009DFCF7A6
:109000005FFB33462A46FCF78DF9FCF79FFBA086F1
:10901000012580B2ED03A84201D3401BA086E08B5E
:10902000FCF74EFB154A164BFCF796FA0646A08E47
:109030000F460090FCF744FB32463B46FCF772F9C2
:10904000FCF784FB80B2E086A84201D3401BE08697
:109050000C4900980968486100982087FEBD00000F
:10906000580100204C0100201904560E2D6240408A
:10907000E17A0000700000201F050000F853E3A50E
:109080009B843E400416002070470000F0B589B074
:10909000002004900A2002F0A5F87D20400102F093
:1090A000BBF8B34800228270C16BB34C491CC1634A
:1090B000B049C38D098A2546C918C1852146C275A4
:1090C00013310791473103916D393135AB4F223060
:1090D00005910290A64E0F21A94871710078207168
:1090E000A84AB079127840001043B27D9200104334
:1090F000E071B08FE070000A2072A17431461E2228
:109100009C310798FCF73AF8402228469E49FCF724
:1091100035F8029903980A7BC274497B01750920CE
:1091200060729A480078A072B08C2073F07D410084
:1091300030469C30091805980A78027549784175BF
:10914000762000228C4902F037F9707906214843D5
:1091500000211C3002F042F9022002F093F80021B5
:109160000F2001F0BFFF38423064F8D0306C411C52
:1091700018D040047ED58122D20100210F2002F0B8
:10918000F0F80021102001F0ADFF41067A48490EA9
:109190000022B43001F0DCFF7748B430417A022974
:1091A00002D0BDE001F0ECF802227949401DFCF745
:1091B00009F80028F5D16E480222C07D41006C48B4
:1091C0009C3009186C48B530FBF7FCFF0028E8D14B
:1091D00002F055F9664AD167906702F03DF9644A9A
:1091E000803203C2049800282CD1012004906248E8
:1091F000684E8C30C08E604930805D488C31098F5C
:1092000041846548FDF7F0FE5949644A0885488C59
:10921000FF30C33080B2488490420CD9524280184B
:10922000488430885D4A401C80B20B3230809042C6
:1092300001D30020308030887D22D20050434A8CF8
:10924000801848654C4869468C30428E0A80808E72
:10925000488049490422B531C81FFF38FBF78EFF0B
:109260004348494AC07D00998000115040498031EF
:1092700003C900E075E0FF235B040022C0185141E0
:109280000906060A0E43304601F0A5FF71084900A1
:109290000A0E0802364900268031CA6088603448C8
:1092A000C36F826F3448483802F0BEF830488030CF
:1092B0000CC83148443802F0B7F82D488030C368F4
:1092C00082682D48403802F0AFF82B49002252390D
:1092D0003C2002F071F800213C2002F07FF80120D0
:1092E00001F0D0FF2249087308468078401C88703E
:1092F00001210520C9030007FCF712FE1C48007B72
:10930000002805D100210F2001F0ECFE0006F9D560
:10931000802200210F2002F024F81548467002E058
:109320001349012048701248C17D491CC9B2C1755A
:109330000F2900D2CEE60498002810D10C4A184913
:10934000908C002802D00B88984201D9088890841C
:10935000144980B20988401E48431349088009B067
:10936000F0BD124A00210F2001F0FBFFD8E70000FA
:1093700070000020280E00205C12002000D027245E
:109380003C01002070010020781400204C010020D6
:10939000600100206C01002004160020E70300009B
:1093A00048010020460100204401002000902724AD
:1093B000F8B532493048086002F044F9304800F00E
:1093C000A3F9304CE0822E48801C00F09DF92083E8
:1093D0002B48001D00F098F960838B212A488900F2
:1093E0004180014640310979284F0906090E617014
:1093F00006D1C7800121C1870A21418700218187C9
:10940000234AC18E1170C18F2171818F6171817A60
:10941000A1708588052165626181C6883046FBF7A9
:1094200067FEA08101462846FBF762FE8800081807
:1094300085B2164825816843FCF742F9154A164B58
:10944000FCF78AF8FCF782F9E081658231463846FC
:10945000FBF74EFE20820146C820FBF749FEE08361
:109460000120A083FCF760FDA082E2890B490C4833
:10947000FDF7BEFDF8BD000075A1000868000020E2
:10948000004F00083C010020E80D0020E803000028
:1094900018000020F853E3A59B843E40FF7F0000A6
:1094A00004160020F8B5754C00202071744D012081
:1094B0002880744EC8203080E07A401CE072C007DB
:1094C00006D0A08C411EA184022801D2C820A0840D
:1094D0000120C043FFF770FD0A2001F083FE7D20CC
:1094E000400101F099FE02216748FDF753FB002877
:1094F0003FD00020654980000978664F4900084345
:10950000634909780843B872102078726248C188AC
:109510007D20C000FBF7ECFD787360485E49007861
:10952000B87338460B308A780270C97841705A494E
:10953000421C20310B7ED370497E11715649D01CDC
:1095400022310B7E5371497E9171534940310A7C1F
:109550000271497C417100223946172001F02CFF2D
:109560000021172001F03AFF022001F08BFE4C4F42
:1095700003E00120BEE7FEF77DFE00210F2001F091
:10958000B1FD38422064F6D0206C411C73D04004F9
:109590006FD58122D20100210F2001F0E2FE0021CF
:1095A000102001F09FFD41063A48490E0022B430D8
:1095B000E16501F0CDFD374FB437787A112858D1E5
:1095C00002223849781DFBF7FDFD002851D1F81F14
:1095D000027A69460A70407A4870B97A2980C820B0
:1095E000FBF786FD3080387BA08438462E4D283826
:1095F000C08E2880394621482839098F41842B485C
:10960000FDF7F2FC2085608C2949FF30C33080B221
:10961000608488420CD949424018608428882449D3
:10962000401C80B20B312880884201D30020288062
:1096300028887D21C9004843618C4018606500F08E
:10964000A3F868460088E0841249B87CC73160718D
:10965000420008460D466930FBF790FD60792946C7
:1096600042001448FBF78AFDA08CFF2801D003209C
:109670002070F8BDFFE700F083FE000070000020BE
:109680004C0100205A01002000040050400100203D
:10969000410100205C120020E80D0020180000208D
:1096A00000D02724600100206C0100200416002057
:1096B000E7030000A413002070B586B014216846AB
:1096C000FBF775FD01250F4EED03002229463046BC
:1096D000FDF76DFA0120002401900294694600957F
:1096E00003943046FDF79AF90320019002946946ED
:1096F000009503943046FDF791F9022001F020F81F
:1097000006B070BD0004005000887047704700002C
:10971000F8B5044600206A461080194D55222A707B
:10972000AA226A700322AA70661DEE702A716971FE
:10973000144A49008918AC712246E81DFBF71EFD4A
:10974000002007E029186A468978128889186A4635
:109750001180401CB042F5DB611DA81CFCF742FAE9
:1097600001466846018029190078C871684640782A
:10977000087221460931024800F012FBF8BD0000D2
:1097800042150020E80D0020FEB5FFF7A1FB25489B
:10979000FDF72AFC244C86B2268560790A21081A36
:1097A000C000FBF779FF07460191A06EFBF788FF29
:1097B0001E4A1F4BFBF7D0FE00900D463046FBF7CC
:1097C0007FFF2B46009AFBF7ADFD3A46019BFBF766
:1097D000A9FDFBF7BBFF85B2A586E08BFBF770FF09
:1097E000124A134BFBF7B8FE06460F462846FBF716
:1097F00067FF32463B46FBF795FDFBF7A7FF81B2BB
:109800000120C003E186814201D3091AE186854225
:1098100001D3281AA0860349A08E096848612087D1
:10982000FEBD00000416002070000020F853E3A5E0
:109830009B843E40034A1168382389B2994301430F
:10984000116070470030014010B5FDF7BDF910BD43
:1098500010B59AB034216846FBF7A9FC14210DA875
:10986000FBF7A5FC1C2112A8FBF7A1FC1B48016813
:109870000324E402A143C21489180160FDF732FCFD
:1098800017480169A143016106200090FF200130C3
:1098900002900120039010200490022009904004BF
:1098A0000B90000100240C900A946846FDF748FED6
:1098B0000F200D9003200E900F941094012111940D
:1098C0000DA8FDF713FD812012900320800418904D
:1098D000149412A8FDF758FC1AB010BD0070004097
:1098E0004010024010480168821511430160C168B0
:1098F0000E4A1140C16001680D4A11400160816843
:109900004908490081600168012292049143016085
:10991000C168FD2212049143C16000210161064922
:109920000448886070470000001002400C40FF8827
:10993000F6FFF6FE0050000800ED00E010B5CB0683
:10994000DB0E0121046A99408C430462016A9A404B
:109950001143016210BD0000F8B5102405252D0744
:10996000AC62AF20800000F0F2FEAC6101F0CEFBF3
:109970002F4C304F304E60670EE001F0C7FB606740
:10998000FEF778FC606C411C6164142804D92BA09C
:1099900000F078FC2D48C760606FB042EDD1002622
:1099A000666420780127FF03030000F0A4FC05048F
:1099B0000C192D303200012239462846FDF7F7F800
:1099C000FFF770FD06E0012239462846FDF7EFF863
:1099D000FFF75CFB002239462846FDF7E8F818E05F
:1099E000607B0122401C607339462846FDF7DFF892
:1099F000FCF7B6FA002239462846FDF7D8F8607B16
:109A0000052806D9267004E0FEF75CFF01E0FFF7A9
:109A10003DFB02210E48FDF7BDF8002805D00020CF
:109A20000C49087001F058FAF8BD0120F8E7000071
:109A3000700000200400FA053001CADE44572049B6
:109A400044204552524F522E0D0A000000ED00E016
:109A5000000400507001002010B5818CC90707D0A8
:109A600001684A6801235B049A43836A1A434A6087
:109A7000818C890707D501684A6801231B049A4332
:109A8000C36A1A434A60818C490707D501684A684E
:109A900001239B049A43036B1A434A60818C090794
:109AA00007D501684A680123DB039A43436B1A43D5
:109AB0004A60818CC90607D50268916801231B039F
:109AC0009943836B19439160818C890607D501689E
:109AD0008A6801235B039A43C36B1A438A60818CB3
:109AE000490612D503685A6801210905046C8A43A6
:109AF00022435A60026C8A4207D1026851680323EC
:109B00005B059943436C19435160818C090607D565
:109B100001684A680123DB04806C9A4302434A606F
:109B200010BD0000F8B50446002680300660FDF741
:109B300045F8054620680068124F000709D5012145
:109B40002B46002249052046009700F0A1FA002884
:109B50000DD12068006840070BD501212B4600225B
:109B600089052046009700F093FA002801D00320D1
:109B7000F8BD2020A067E0672666603426750020C7
:109B8000F8BD0000FFFFFF01F8B5154CC826E078CE
:109B9000002823D16079002820D101206071114D67
:109BA000686B0027002818D0686BC821081A0FE0DE
:109BB0000D48E168405C61698847E068401CE060EE
:109BC000E068C82800DBE760696BC820401A761E91
:109BD000E168814201D0002EEADC6771F8BD000027
:109BE0005400002000000240200D002070B5224CDF
:109BF000E07800283FD1207900283CD10120207155
:109C00001E4EF16900250906002933DA21566257F4
:109C100091420AD1F06940062CD5A079002829D0BC
:109C2000A5712089401C208124E0A179002903D15D
:109C3000A0710A2000F08BFD00202056CC21484363
:109C40000F494218206912181279B262401C002292
:109C50002061A256CC235A43895881420ADC2561EF
:109C60002078401C207020780E2800D12570A07824
:109C7000401CA070257170BD5400002000380140C8
:109C8000F801002010B5806A0022014640314A8365
:109C90004A82FDF76BFF10BD70B5846AA06FE56F57
:109CA0002168896800260906002906DA212804D1DE
:109CB00052200653204600F06BF82068806840066A
:109CC00006D5222D04D15A200653204600F047F82D
:109CD0002046803001681022114301602046FDF7C4
:109CE00045FF70BD10B501460968806A096889069C
:109CF0001CD400225A210A5201680A68FF2301334A
:109D00009A430A6001688A68520852008A600168B2
:109D10008A6840239A438A602021C167016E012925
:109D200004D101680A6810239A430A60016E012970
:109D300002D0FEF7FDF810BD5821095AFDF714FFB7
:109D400010BD10B5806A016E012902D0FEF7F1F84E
:109D500010BD5821095A4908FDF706FF10BD0168DA
:109D60000A68FF2321339A430A6001688A6852080F
:109D700052008A60016E012904D101680A6810232B
:109D80009A430A602021C16700210166416670473D
:109D900001680A68C0239A430A60202181677047DE
:109DA00070B5164CE278002A0CD12279002A09D12C
:109DB0000122E2700025C82903DC0222A256002AF3
:109DC00001DCE57070BD0123E356CC2253430C4AFD
:109DD000D1500123E356CC2673439B180A46014613
:109DE000181DFBF7CBF96078401C607060780E2876
:109DF00000D16570A078401EA070E2E754000020FA
:109E0000F8010020F8B50446016880682369E66916
:109E100018436369002533431843724A0B68724E36
:109E2000334003430B602168486803231B039843B6
:109E3000E368184348602168A069914201D0236A11
:109E400018438B680B263602B34303438B60674984
:109E5000236867488B420CD1C0688007800F06D00A
:109E6000012839D0022835D0032821D11EE001274E
:109E70001FE060498B420AD1C0680C21084027D0FE
:109E8000042829D0082825D00C2811D10EE09342AF
:109E90000ED1C16803208002014019D00120800248
:109EA000091A19D0091A15D0814201D1082700E0FA
:109EB00010274F49504840398600934232D1002F35
:109EC0000CD0022F0DD0042F10D0082F7FD126E008
:109ED0000027EEE70227ECE70427EAE7FDF7D4FACC
:109EE00006E00968C90605D4304603E0FDF7ECFA40
:109EF000002872D0626851005118814267D811035E
:109F0000814264D3010E06025008002330185941E3
:109F1000FBF704F903210902411A384A55E00120F0
:109F2000C003E7E70122E369D20393422BD13B0050
:109F300000F0E1F90906090C4D114D4D4D274D007A
:109F4000FDF7A2FA09E0FDF7AFFA06E00968C906D5
:109F500005D4304603E0FDF7B7FA00283DD061682C
:109F600040004A088018FBF7C3F880B20146244A33
:109F7000103991422BD8511C01400007400F084373
:109F800029E01046EBE73B0000F0B5F90906090CA3
:109F90002112212121232100FDF776FA0AE0FDF7A5
:109FA00083FA07E00968C90606D4304604E00EE0EB
:109FB000FDF78AFA002810D061684A081018FBF7EC
:109FC00097F880B201460E4A1039914203D9012513
:109FD00003E01046F0E72168C86000206066A066D4
:109FE0002846F8BD00480040F369FFEF0038014003
:109FF000401002400044004000093D00FFFC0F00FB
:10A00000EFFF0000F8B504464165403000262746C2
:10A01000028380373E602220E0672546206F60354E
:10A0200000281CD01749C162216F17480863216FAF
:10A0300016484863206F8663236F606D9C46134605
:10A040002168024660462431FCF710FC002806D047
:10A05000102038602E752020A0670120F8BD2E75D5
:10A0600020680168FF220132114301602068816885
:10A070000122114381602068816840221143816080
:10A080000020F8BDE59C0008439D0008999C00084D
:10A09000FFB581B005460F46044660350A9E39E09B
:10A0A000701C37D0FCF78AFD0499401AB04222D8C0
:10A0B000002E20D02068016849072BD5C069C04315
:10A0C000000527D401202168C002086220680168C9
:10A0D000FF22A1329143016020688168490849004C
:10A0E00081602020A067E067803420600020287510
:10A0F000032005B0F0BD20680168FF22A132914322
:10A100000160206881684908490081602020A067BB
:10A11000E067EBE72068C1693846884305D0002135
:10A1200003988142BCD00020E3E70121F8E700005A
:10A1300010B504491020096808620248FDF718FDAF
:10A1400010BD0000CC16002001490D20887070471A
:10A150005400002010B5FEF7B3FAFEF78BFBC822BF
:10A1600002490348FDF7B4FE10BD0000200D002099
:10A17000CC160020F8B53E4C002321783D4A1D4600
:10A18000082910D0072947D0062950D0052952D0D8
:10A19000042953D0032954D0002956D0012958D07E
:10A1A00002295AD05BE0A17800264A1F04E0314F13
:10A1B000BF5DFB189BB2761C9642F8DB6679277967
:10A1C0009A195118E3786278C9188918C919401882
:10A1D000C0430006000E1AD1012E14D0022E16D153
:10A1E00025482449C018FAF7C9FF01F087FF642009
:10A1F00000F0A6FABFF34F8F21492048C860BFF393
:10A200004F8F00BFFDE759081046FFF781FA257010
:10A21000E570A570A571F8BDA1795054491CC8B26C
:10A22000A071A178491F8842F5D1082001E0607033
:10A2300007202070F8BDE0700620FAE76071052065
:10A24000F7E7A070E5700420F3E7552807D1012057
:10A25000EFE7AA2803D10220EBE7032803D02570FB
:10A26000E570A570F8BD032020702071F8BD0000D6
:10A2700034010020DE140020E80D00200400FA055F
:10A2800000ED00E010B5024A024900F0E5F910BD0A
:10A2900041B40008880100202021020C01D01021C7
:10A2A0001046020A01D010460839020901D01046B2
:10A2B000091F820801D01046891E420801D0881E5D
:10A2C0007047081A7047F8B5040C8BB2264682B264
:10A2D0005E430D0C1046370C58433604801900219C
:10A2E000794116466E43370C36048019794126466B
:10A2F0006E438919F8BD30B47446641E2578641C19
:10A30000AB4200D21D46635D5B00E31830BC1847CA
:10A310004900CA020243100000D004204A0D01D0B7
:10A3200001221043044A490D914201D10221084300
:10A33000012800D105207047FF0700008307FF2296
:10A34000DB0E9A408907090E9940002808DB830834
:10A3500009489B001B181868904308431860704711
:10A360000007000F0838830804489B001B18D869B1
:10A3700090430843D861704700E400E000ED00E03E
:10A38000BFF34F8F04490348C860BFF34F8F00BF2E
:10A39000FDE700000400FA0500ED00E0F8B5044612
:10A3A0004F1EC8000838211815461E46086849681F
:10A3B0003A4606239A4310D02A463346FBF764F800
:10A3C0003A46D200083AA3181A687F1E5B68FAF76B
:10A3D000A9FF06223B469343EED1022F23D0042F40
:10A3E00011D0062F2FD12A463346FBF74DF8E36AEA
:10A3F000A26AFAF797FF2A463346FBF745F8636AE5
:10A40000226AFAF78FFF2A463346FBF73DF8E369E5
:10A41000A269FAF787FF2A463346FBF735F86369E6
:10A420002269FAF77FFF2A463346FBF72DF8E368E7
:10A43000A268FAF777FF2A463346FBF725F86368E8
:10A440002268FAF76FFFF8BD002210B513461046D8
:10A450000149FBF781F810BD0000F03F10B5FAF795
:10A4600061FF10BD002210B5134610461146FBF7E0
:10A4700073F810BD10B50721024A00200907FBF749
:10A48000E3F810BD01030000034A10B500201107D6
:10A49000FBF7DAF810BD000001FDFFFF02E008C87D
:10A4A000121F08C1002AFAD170477047002001E04E
:10A4B00001C1121F002AFBD170470000014908604A
:10A4C000704700008C01002008B50021684601702B
:10A4D0006B46012202212C2000F052FF0221684627
:10A4E00001706B4601222C2000F04AFF08BD0000DD
:10A4F00038B504466D20694608706B46012207494D
:10A500002E2000F03DFF0649002C01D0054A00E056
:10A51000054A2E2000F01AFF38BD00000608000092
:10A5200006180000070600000716000038B50446AC
:10A530006B4602220021362000F0EEFDB3212300FD
:10A54000FFF7D9FE0E0F08153A3A3A3A1C273A3A65
:10A550002F34483A0021684601704078410849008C
:10A5600014E06946087880088000401C04E06946D1
:10A57000087880088000801C08701DE0684602781A
:10A580000A40483202704178802001436846417099
:10A5900012E0684602780A40027040784106490E8F
:10A5A000F4E7694648780221084303E069464878A1
:10A5B000FD210840694648706B4601220021362083
:10A5C00000F0DEFE012200AB11463620013300F020
:10A5D000D7FE38BD69460878CF210840694620304B
:10A5E000CAE708B5032168464170012101706B4636
:10A5F00002220021362000F0C3FE0122D2030621F0
:10A600002D2000F0A3FE012000F09AF80120FFF7B2
:10A610008DFF08BD08B5020A69464A7008706B468E
:10A62000022204212D2000F0ABFE032069460870B1
:10A630006B46012206212D2000F0A2FE0020694673
:10A6400008706B46012206212D2000F099FE0A2198
:10A650002D2000F047FD08BDF8B516460F4604460C
:10A66000002503E03946B047641C6D1C20780028A3
:10A67000F8D12846F8BD0000F8B54A002B4B520D22
:10A68000D6182B4A0C460546142E2BDA002E12DA69
:10A69000284BFAF747FE00221346FBF79DF840D2FD
:10A6A000002C03DA0124E40700253AE02046284381
:10A6B00037D0214C14E0214F0B46F7403B402B4351
:10A6C00031D01C4BFAF72EFE00221346FBF784F81C
:10A6D00027D2002C03DD01200005F0400419BC4303
:10A6E00000251EE0332E1EDC33460027143BFF43BB
:10A6F000DF40384217D00F4BFAF7BEFE0022134658
:10A70000FBF76AF80DD2002C0ADD142E0CD0342091
:10A71000811B012088404019A84200D2641C0546D4
:10A72000BD4321462846F8BD641CF9E701FCFFFF44
:10A730009C7500883CE4377E0000F03FFFFF0F006F
:10A740007D2110B5C900484300F001F810BD00217B
:10A7500040E000BF00BF00BF00BF00BF00BF00BFA0
:10A7600000BF00BF00BF00BF00BF00BF00BF00BFF1
:10A7700000BF00BF00BF00BF00BF00BF00BF00BFE1
:10A7800000BF00BF00BF00BF00BF00BF00BF00BFD1
:10A7900000BF00BF00BF00BF00BF00BF00BF00BFC1
:10A7A00000BF00BF00BF00BF00BF00BF00BF00BFB1
:10A7B00000BF00BF00BF00BF00BF00BF00BF00BFA1
:10A7C00000BF00BF00BF00BF00BF00BF00BF00BF91
:10A7D00000BF491C8142BCD37047FFB581B01E4603
:10A7E0000F46040026D00B9903980143A06A394311
:10A7F000826807209047002818DB0A99A06A314335
:10A80000826806209047002810DB25462035A9796C
:10A81000032F01D908200143032E01D9042001434D
:10A82000A06A826809209047002806DA0120C04308
:10A8300005B0F0BD0020C043FAE7384600F000F94B
:10A840002060304600F0FCF860600A986870039859
:10A85000A870EF702E710B9868710020E8E7000077
:10A86000F7B50446002090B000900190002C05D070
:10A870006A46062101F07CFC062803DA0020C0436A
:10A8800013B0F0BD684640780102684600780004C5
:10A890000918684680780818FAF712FF05466846D6
:10A8A0000391007901026846C078000409186846DF
:10A8B00040790818FAF704FF032206460F4692076C
:10A8C0005C4BFAF789FF07D200225B4B30463946D2
:10A8D000FAF7CCFD06460F4603229207554B284651
:10A8E0000399FAF779FF07D20022534B28460399C0
:10A8F000FAF7BCFD054603912068FAF7E1FE02462F
:10A900000B4630463946FAF727FE07460A200791DC
:10A91000205EFAF7C1FE3A46079BFAF7B5FD0646F8
:10A9200008200991205EFAF7A5FE0021C943FAF735
:10A93000EDFCFAF729FF3246099BFAF7F3FC069182
:10A9400008906068FAF7BCFE02460B462846039959
:10A95000FAF702FE05461A200E46205EFAF79CFE24
:10A960002A463346FAF790FD0C9009911620205E96
:10A97000FAF792FE099B0C9AFAF7D4FC05910A901B
:10A980002A46334638460799FAF77EFD059B0A9A10
:10A99000FAF77AFD05910A901420205EFAF77CFE02
:10A9A0003A46079BFAF770FD07461C200791205E88
:10A9B000FAF772FE2A463346FAF766FD0E900B91BF
:10A9C0001820205EFAF768FE0B9B0E9AFAF7AAFC95
:10A9D0002A463346FAF758FD0B910E902069FAF794
:10A9E0005BFE0B9B0E9AFAF79DFC2A463346FAF75C
:10A9F0004BFD05460E46E068FAF74EFE2A46334602
:10AA0000FAF790FC3A46079BFAF78CFC059B0A9AEA
:10AA1000FAF788FC01229207084BFAF735FD024647
:10AA20000B46129C0898069903C411980CC000208C
:10AA300026E70000FFFF5F4100007041E17A843F9C
:10AA400000B50121C9040300FFF755FC081A0508E9
:10AA50000B0E1114171A0320C00400BD0720C004F8
:10AA600000BD0F20C00400BD1F20400300BD3F20DB
:10AA7000400300BD7F20400300BDFF20400300BD18
:10AA8000084600BDFEB5264F0D4604000FD0002D30
:10AA90000DD0264600202036B071F07129680D20B7
:10AAA0008847002801DA7800FEBD102801D038461A
:10AAB000FEBDA562E968002901D02820884720460C
:10AAC00000F030F80028F3DBA06AA52182680E2090
:10AAD0009047A06A962182680F209047A06A0221C1
:10AAE000826862209047A06A002182680E20904709
:10AAF000A06A002182680F2090477179302001916F
:10AB000000900623202201212046FFF766FE002840
:10AB1000CEDB204600F0AEF80028C9DB0020FEBDE9
:10AB2000FFFFFFFF10B586B0044614216846FAF710
:10AB30003EFB002C7ED0A06A122143686A4610209A
:10AB40009847122877D168460078012201016846AB
:10AB5000407812030009081843492081884201DD2A
:10AB6000801A20816846837840780007000D181805
:10AB70006081884201DD801A608168460079012287
:10AB800001016846C078120500030918684640793B
:10AB9000000908183549E060884201DD801AE0604C
:10ABA000684640790007030B6846807900021B184D
:10ABB0006846C07918182061884201DD801A20613A
:10ABC0006846417A007A0002081802B2284801213A
:10ABD0000904A282824201DD521AA2826A46D37A15
:10ABE000927A12029A1812B2E282824201DD521A5D
:10ABF000E2826A46537B127B12029A1812B22283B7
:10AC0000824201DD521A22836A46D37B927B120272
:10AC10009A1812B26283824201DD521A62836A4636
:10AC2000537C127C12029A1812B2A283824204DD73
:10AC3000501A01E00BE008E0A083A06A0168282018
:10AC40008847002806DA0120C04306B010BD002066
:10AC5000C043FAE7C011C0072034002800D080208C
:10AC600060710020F1E70000FF070000FFFF070010
:10AC7000FF7F000010B5040009D0A06A0721826898
:10AC800008209047002805DA0120C04310BD0020AD
:10AC9000C04310BD072020342070002010BD0000EC
:10ACA000FEB5044600200190009060797349400091
:10ACB0000E5A61782578491E7148CFB20163042D80
:10ACC00077D0072D75D000210291217801736C494E
:10ACD000E379012292058969002B6CD0914381614F
:10ACE0006748217A4173217A82698907890B0A436F
:10ACF00082610021042000F034FB324661492E209D
:10AD000000F024FB3846FFF7F3FB5F4E0522705D31
:10AD1000810040185D49431807212B2000F030FBCB
:10AD20005B49029801220B180B21282000F028FB18
:10AD3000705D584980000A580C21282000F011FB52
:10AD4000E079554980004018A1794900425A022112
:10AD5000272000F0FBFA51487E00825B0421272067
:10AD600000F0F4FAE079002829D0A07804282CD04B
:10AD700028206946087220220621272000F0E6FAE2
:10AD800002AB01222621272000F0FAFA44493801BB
:10AD90004018E178890042580821272000F0E1FAA4
:10ADA000A17A601C627A0902114313D016E000E018
:10ADB00001E0012188E71143F608816190E76422F0
:10ADC0000621272000F0C2FAE0E710206946087249
:10ADD0000246D1E733490172090A4172417A007A89
:10ADE0000A0202432021272000F0B0FA2E4F0C2146
:10ADF00023203A6800F0B5FAF01982880421232054
:10AE000000F0A4FAA07900280BD0E07927490122AC
:10AE100043180021212000F0B3FA03200190012003
:10AE200000902A07120F100102436078002180076A
:10AE3000000B0243019800050243009840040243BE
:10AE40002079C006400902436079C00602431F20F2
:10AE500000F087FAA07861780123084302040848CB
:10AE6000DB030261E179490319430A4302610021CE
:10AE7000082000F076FA0020FEBD0000A4C2000801
:10AE8000BC010020042800004CC20008240000205F
:10AE90004200002054C2000874C2000880C20008AA
:10AEA00084C20008411000006CC200084400002069
:10AEB00038B50C4607498A8B002102432C2000F04C
:10AEC00045FA684604706B46012206212C2000F0EA
:10AED00057FA38BDBC01002010B5FFF7F5FA10BDD8
:10AEE00010B504460421362000F0FCF80121C90207
:10AEF000002C01D0084300E088430246042136209C
:10AF000000F02FFA10BD000038B5402069460870E7
:10AF100000210E2000F0E6F80446002211460E2023
:10AF200000F01FFA6B46012200210D2000F028FAE4
:10AF3000074A00210F2000F014FA00F0EDF9224634
:10AF400000210E2000F00DFA02480021017338BDE7
:10AF5000F8FF2724DC010020FEB5054604206946E1
:10AF60000870514C002060752146203120634871E3
:10AF70000873A0836063A06300F0C8F84B4E2060A4
:10AF800002E000F0C3F82060B042FAD10020FFF7E1
:10AF9000CDFA00F0BBF8464E20603078242801D965
:10AFA000243806E00621FAF7A3F80622101A400119
:10AFB0000843020601040A4301020A430243B26045
:10AFC000706000211E2000F0CCF900F09FF8206096
:10AFD0006B4601220021242000F0D2F91E20FFF749
:10AFE00019FB86B2300AA0730420FFF713FB074653
:10AFF00000F08CF820603806000E0DD00220694663
:10B00000087101AB012212212D2000F0B9F9A08BAB
:10B01000012109030843A08300F078F8206006208E
:10B02000FFF7F8FA60600720FFF7F4FAA060F00677
:10B03000C00E207501D110202075C0B200F0DCF9DF
:10B04000E80707D0FFF7CDFAA08B0121C90208431A
:10B05000A0830AE00521362000F02EF815490840AB
:10B0600002460521362000F071F90120FFF75EFA53
:10B070000021042000F036F8A0610021262000F015
:10B0800031F815218903084302460021262000F0EB
:10B0900068F900222621362000F058F900F036F831
:10B0A00020600020FEBD0000BC0100203001CADE8F
:10B0B00018000020FFFD000038B5094C89B280B2AD
:10B0C0006B46022200F028F8002806D16846407836
:10B0D000010268460078081884B2204638BD000096
:10B0E000FFFF000038B50024E44389B280B26B460C
:10B0F000042200F011F8002806D103216846435CC1
:10B100002202D418491EFAD5204638BD10B50021B8
:10B110000846FFF7E7FF10BD38B5002909D04024E5
:10B1200020436C462070C8B27F2906D86070022088
:10B130000AE069460870012006E0802420436C463E
:10B140006070C809A0700320694600F0B1FF38BDE7
:10B1500010B5144603460A4621461120FFF7DCFFCE
:10B1600010BD10B50346052200211520FFF7D4FFBE
:10B1700010BD10B50346052200211720FFF7CCFFB4
:10B1800010BD38B5054600206946087000F0C4F8C7
:10B19000FF2401342246002D01D003221202002197
:10B1A0000D2000F0D3F8002D13D06B4601220321AF
:10B1B0000F20FFF7B1FF68460078000709D5FFF7B9
:10B1C000A3FE224600210D2000F0C0F80020C0435D
:10B1D00038BD002038BD10B5024601210A2000F01C
:10B1E000C0F810BD10B5044600211A20FFF77AFF01
:10B1F000000D22030005120B024300211A2000F06B
:10B20000B0F810BD10B5024602492E2000F09EF89D
:10B2100010BD000004180000F8B505466B46012279
:10B2200003210420FFF778FF0126114C3607002D7B
:10B230000DD02A4600210C2000F088F869460878D5
:10B240001021084369460870A069304307E0694649
:10B250000878EF21084069460870A069B0430B46A2
:10B26000A06101220321042000F08AF8F8BD00004B
:10B27000BC01002010B502460021182000F066F83D
:10B2800010BD0000F8B50746002568460570B807F0
:10B29000204C2E4600280ADA8020694608706B464A
:10B2A000012200210D2000F06BF801202073F80727
:10B2B0006946087821D006210843694608706B4624
:10B2C000012200210D2000F05BF803210F20FFF781
:10B2D000F3FE8121C900084219D040206946087058
:10B2E0006B46012200210D2000F04AF80020FFF7F4
:10B2F000F7FD00252673ED4309E002210843694666
:10B3000008706B46012200210D2000F039F8284614
:10B31000F8BD0000DC0100201CB56B4601220321B2
:10B320000F20FFF7F9FE684600784022C10910405F
:10B33000C9014000814208D00120694608710246D7
:10B3400001AB03210D2000F01BF81CBD08B56B46B6
:10B350001A70120A5A7089B280B2022200F010F8F4
:10B3600008BD38B500236C46E254120A5B1C042B5E
:10B37000FADB89B280B22346042200F001F838BD1E
:10B3800038B58024002909D0C02528436D4628708F
:10B39000C8B27F2907D86870022009E020436946B7
:10B3A0000870012004E020436870C809A8700320D9
:10B3B000694600F027FF38BD10B514460123121866
:10B3C0009B029A4202D90020C04310BD0B46821E48
:10B3D00021460920FFF7D4FF002010BD10B5054A13
:10B3E0008905126901430A4300210820FFF7B9FFCC
:10B3F000002010BDBC01002038B504466B46012278
:10B400000E212B20FFF788FE68460078E1064009F0
:10B410004001C90E0143684601706B4601220E21AE
:10B420002B20FFF7ADFF38BD10B5002142541C069C
:10B43000120A22431B0A491C0429F7DB10BD000035
:10B4400013B501231A4669460248FCF773FD0098BC
:10B450001CBD0000CC1600207CB5002425466846A3
:10B46000FFF77FFE04206946220E2D0215432202BB
:10B470000C5C1443401EF7D5204629467CBD7CB5A4
:10B48000002425466846FFF774FE04206946220E14
:10B490002D02154322020C5C1443401EF7D52046B2
:10B4A00029467CBDFBF798FBFEF7D2F9FDF71CF9A6
:10B4B0003E493F48002522C005608561C5613D4980
:10B4C0000562C1600838FBF719FDFDF7F9F8FDF7D3
:10B4D000D1F9FDF7ADF9FDF7BFF8052401222407E6
:10B4E000D1032046FBF763FBFDF762FFFCF79CFFEF
:10B4F000FAF754FBFAF7D6FBFAF7A4FBFCF79CFD2E
:10B500000721A015FFF7D4FCFFF7E6FC0122110389
:10B510002046FBF74CFB2648C8222749C830FCF7D9
:10B52000D7FC264F264E274C387800280FD130788C
:10B53000002801D003280AD10121C9022248FBF7C3
:10B5400029FB002803D101210846FBF7EBFDE07839
:10B55000002828D06078002825D0E57072B62078C1
:10B560000F280AD90120184900038861FEF7F4F971
:10B5700001201549000388620CE0012251031248A2
:10B58000FBF715FBFEF7E8F90121002249030E48FD
:10B59000FBF70DFB62B6FCF76DFE208C0028C3D0D4
:10B5A000401E2084C0E7FCF765FEBDE7007C00403C
:10B5B00004160020FFFF0000200D00205A0000208C
:10B5C000840000203C0100200004005010B586B02B
:10B5D0001748FBF716FC14216846F9F7E8FD1548F3
:10B5E000009003200190002002900520694600078A
:10B5F000FBF714FA69461048FBF710FA69460F4842
:10B60000FBF70CFA01210846FBF78CFDFF240134FF
:10B610002046FBF75FFD0A490868042210430860D2
:10B620002046FBF767FDFBF76DFD06B010BD00007F
:10B6300004160020FFFF0000000400500008005026
:10B640000070004010B50122920217491748FAF71E
:10B65000ADFB1548164902888A4223D00180042197
:10B660008180FF21F531C1800A21018100211E2244
:10B670004181D24382810122C28181834323C386D7
:10B6800002230387782343878287C287024640329A
:10B69000118451849184C183918014238382118207
:10B6A00000F02CFD10BD0000E80D002000FC00089B
:10B6B000AA550000F0B51FB496B084460C46024669
:10B6C000199D1898039049006800630049084008D4
:10B6D0000193002A01D0012600E000269E19FE4BAE
:10B6E000F6185B109E422BD36E00039F0296002F2C
:10B6F00000D00127F719F84EF84BBE199E421FD310
:10B70000039E0346F64F334309D03B469C4201D18A
:10B71000002A04D0019B002A05D0012604E0002065
:10B7200039461BB0F0BD00269E19EE4B9E4207D84D
:10B73000039F029E002F00D00127F6199E4207D9D1
:10B740002B4660462146189AFEF788FE1BB0F0BDD6
:10B750000023002C29DAE44EB04226DAE34EB04250
:10B7600001DB022321E0DE4EB0421EDBE04E070D7E
:10B77000BE19142E09DD3427BF1B039EFE4001961F
:10B78000BE40039FBE420BD00FE0039F002F0CD1A1
:10B790001427BF1B0646FE400196BE40864204D1D8
:10B7A000019BDE07F60F02239B1B0E46164318D1A2
:10B7B000002D16DA002C03D0022B01D0012B06D06D
:10B7C0000220FEF77BFEFEF73FFE1BB0F0BD02201D
:10B7D000FEF774FEFEF738FE0122D20751401BB07F
:10B7E000F0BD039E002E61D1BF4EB04220D1C148B2
:10B7F000844201D1002A08D0B948814209DB002DDA
:10B8000010DB189829461BB0F0BD0020B4491BB0CE
:10B81000F0BD002D06DA01222946D20718985140C2
:10B820001BB0F0BDB4497944086849681BB0F0BD4D
:10B83000AB4FB84225D1002D1FDA002904D0B14208
:10B8400012D1002A09D018E0002A72D1A649E20FCD
:10B850000020D20711431BB0F0BD0020E20F0146CB
:10B86000D20711431BB0F0BDB14206DA23460020D7
:10B870003946F9F771FE1BB0F0BD104621461BB0EA
:10B88000F0BDB14212DA0126B607B54203D1234614
:10B8900010461946FEE3994EB54207D1261E05DB38
:10B8A0001046314600F040FC1BB0F0BD67007F0839
:10B8B0001646002A40D100290AD08B4A914229D14C
:10B8C000002C0EDD002D1CDB002011461BB0F0BD4E
:10B8D000022B16D0002C14D0012B12D1002C14DB1B
:10B8E0000FE0002C28DA002D09DB012B03D000200B
:10B8F0007D491BB0F0BD002081491BB0F0BD012B7C
:10B9000003D0002001461BB0F0BD00200121C90773
:10B910001BB0F0BD724A91420ED1002C01DA002B0F
:10B9200017D0022B06D00020C043F9F7B5FE1BB09C
:10B93000F0BD90E20120F8E7E217521C94461A434A
:10B9400007D000220892664C62465B1E1A4307D05D
:10B9500009E00120FEF7B2FDFEF784FD1BB0F0BD4B
:10B960000022644C0892674A90427DDD664B674A2C
:10B9700098421FDD914202DC002D05DB4DE0584866
:10B98000814217DB002D48DD0220FEF797FDFEF710
:10B9900071FD05460E460022534B21460898F9F7E3
:10B9A00073FD084671004908C00FC00701432846CF
:10B9B0001BB0F0BD914215DA002D2EDA0220FEF701
:10B9C0007DFDFEF757FD05460E460022464B2146FB
:10B9D0000898F9F759FD72005208C80FC0070243D2
:10B9E000114617E03E4B994223DD002D15DD022064
:10B9F000FEF764FDFEF73EFD05460E4600223A4B7B
:10BA000021460898F9F740FD084671004908C00F23
:10BA1000C007014328461BB0F0BD0220FEF74EFDD3
:10BA2000FEF732FD49004908E20FD20711431BB06F
:10BA3000F0BD002230463946F9F718FD01220546CF
:10BA40000E46D243F9F700FE314A324BF9F714FDA6
:10BA50002A463346F9F718FD0022284BF9F70CFD6A
:10BA600007462A46334600E064E003911046194633
:10BA7000F9F70AFD3A46039BF9F706FD074603224C
:10BA800009915207244B28463146F9F7FDFC0791EE
:10BA90000C90224A204B38460999F9F7F5FC0746E5
:10BAA00001911F4A1F4B28463146F9F7EDFC3A46F3
:10BAB000019BF9F7DBFC07460B4602460991079903
:10BAC0000C98F9F72FFC00250E462846079B0C9A88
:10BAD000F9F7CCFC3A4627E0FFFF1F00FFFF0F00FD
:10BAE0000000F03F0000E0FF0000F07F0000404356
:10BAF00001FCFFFF0000F0BF560B00000000E03F1C
:10BB00000000F0FF0000E0410000F043FFFFEF3FC6
:10BB1000555555555555D53F4715F73FFE822B6571
:10BB200044DF5DF80BAE543E099BF9F7A5FC0246D5
:10BB30000B4652E1012500202D05A94207DA3522E6
:10BB400030463946F9F780FD06463420C0430A15D1
:10BB50001218FE48101803900803FD49000B01431A
:10BB60000F46FC49884201DC002003E0FA49884284
:10BB700002DA0120119005E0002011900398401C8A
:10BB80007F1B039011980597C200F4480F927844E8
:10BB9000801843680268394630460D930292F9F7DF
:10BBA00065FC07910C9030460D9B029A0599F9F7B8
:10BBB000B9FB02460B460020E549F9F7CDFC099197
:10BBC0000490079B0C9AF9F75FFC129000201090EC
:10BBD000E3480D46784400680E900121781049072B
:10BBE000084311990D9B890440180121C904471885
:10BBF0003946029A0E98F9F739FC3246059BF9F757
:10BC00003BFC02460B4629461098F9F73DFC0646D8
:10BC100002913B4629460E9A1098F9F735FC079B8E
:10BC20000C9AF9F729FC3246029BF9F71FFC099B95
:10BC3000049AF9F729FC0591129A0A902B461046AE
:10BC40001946F9F721FC06460246C6480F460B4640
:10BC500006217844FEF7A2FB32463B460091049051
:10BC600010461946F9F710FC009B049AF9F70CFCF2
:10BC700006460F462B461946129A1098F9F752FBC2
:10BC8000059B0A9AF9F700FC32463B46F9F74AFB56
:10BC9000109A079104902B4610461946F9F7F4FBC9
:10BCA000B14E0022334609910290F9F73BFB079B06
:10BCB000049AF9F737FB0020074602463346009105
:10BCC000F9F7D4FB099B029AF9F7D0FB079B049A7A
:10BCD000F9F7D2FB06460D913A462946009B10988B
:10BCE000F9F7D2FB07910C902B463046129A0D992A
:10BCF000F9F7CAFB05460E463A46009B05990A9895
:10BD0000F9F7C2FB33462A46F9F70CFB02460B460D
:10BD10000746099107990C98F9F704FB00250E4690
:10BD20002846079B0C9AF9F7A1FB3A46099BF9F7BD
:10BD3000A3FB07460722099152078C4B3146284640
:10BD4000F9F7A2FB07910090894A884B3846099978
:10BD5000F9F79AFB07460191864A874B31462846F8
:10BD6000F9F792FB3A46019BF9F7DCFA834B7B44E7
:10BD70000F9A9B181A685B68F9F7D4FA0290099138
:10BD80000398F9F789FC05910490099B029A079999
:10BD90000098F9F7C7FA7A4B7B440F9A9B181A68F8
:10BDA0005B6817460393F9F7BDFA059B049AF9F708
:10BDB000B9FA0E462846059B049AF9F757FB3A460E
:10BDC000039BF9F753FB079B009AF9F74FFB099B7D
:10BDD000029AF9F751FB02460B46199900200C9084
:10BDE0000F461898F9F750FB029104903B460C9AC5
:10BDF00019991898F9F73AFB2A463346F9F744FBA4
:10BE0000029B049AF9F78EFA09910E902A4633465E
:10BE100039460C98F9F738FB06460F46099B0E9AEF
:10BE2000F9F780FA574A0D46914220DB5242AA1890
:10BE3000024310D132463B46F9F718FB04900391B8
:10BE4000514A524B09990E98F9F76CFA039B049AE0
:10BE5000F9F7C2FC1ED20220FEF730FBFEF70AFB08
:10BE600049004908E20FD20711431BB0F0BD6A0038
:10BE7000474B52089A420DD3464AAA18024300D0B3
:10BE8000CBE532463B46F9F7F1FA099B0E9AF9F7F2
:10BE9000A3FCF5D96800002340082C490393020D48
:10BEA0003D4B5218984223DD01200005521CD04022
:10BEB00042195000400D401838497944096813462A
:10BEC0008C463749C1408B4312030121120B0905EF
:10BED00051181422101AC1400391002D01DA484272
:10BEE0000390624630463946F9F7C0FA06460F46D7
:10BEF00032463B4609990E98F9F714FA00252A466E
:10BF0000284B28460591F9F7BFFA07910C90264A6D
:10BF1000264B28460599F9F7B7FA00910290324668
:10BF20003B4628460599F9F7A1FA099B0E9AF9F7BD
:10BF3000A3FA1F4A1F4BF9F7A7FA009B029AF9F7D9
:10BF4000F1F907460B460246099135E001FCFFFF77
:10BF50000000F03F8E9803007AB60B0066070000E1
:10BF6000A8070000D20600000000084009C7EE3F05
:10BF7000FD033ADCF5015B14E02F3EBEA605000090
:10BF80006C05000000009040FE822B654715973C31
:10BF900000CC904000346F3F0000E03FC20400003E
:10BFA000FFFF0F00432EE63F396CA80C615C20BEFA
:10BFB000EF39FAFE422EE63F07990C98F9F7B2F9ED
:10BFC00005460E46079B0C9AF9F750FA3A46099B2C
:10BFD000F9F752FA09912A4633460E90104619464F
:10BFE000F9F752FA074602462F480B4605910521FC
:10BFF0007844FEF7D3F93A46059BF9F745FA2A4605
:10C000003346F9F739FA0746019128463146099B2C
:10C010000E9AF9F739FA099B0E9AF9F783F9012379
:10C0200004910C9000229B0738460199F9F71EFAFB
:10C0300005910E903A4628463146019BF9F724FABD
:10C04000059B0E9AF9F788FA049B0C9AF9F70EFAF9
:10C050002A463346F9F70AFA0022144BF9F70CFA8C
:10C06000064603980D46000541190915002912DC02
:10C0700030462946039AF9F7E7FAFEF749F904280A
:10C0800001D1FEF701FA30462946039AF9F7DCFAA6
:10C09000064601E004E029180B463246214608987E
:10C0A000F9F7F2F91BB0F0BD640300000000F03FA7
:10C0B000F0B58C4600251026052109078E620E4C2E
:10C0C00008E067467F5DE760A768FF07FCD0E76888
:10C0D0001F706D1C8542F4DB0020074606E0E76018
:10C0E000A568ED07FCD0E5681D54401C9042F6D3CE
:10C0F0008E610020F0BD00000030014070B572B6C6
:10C100000124074DA40221462846F9F735FE0028F0
:10C1100004D0224603492846F9F7D2FE62B670BD24
:10C1200000FC0008E80D0020F8B506460C46F9F7BB
:10C1300061FC051E0F4600D00120014349000B4859
:10C140004908411AC90F0DD0002E01D0012100E08D
:10C1500000210C4361004908401AC00F02D10120A0
:10C16000FEF7ACF928463946F8BD00000000F07F24
:10C17000F8B515460E460746002407E03819C0B248
:10C1800000F008F8641C2870E4B26D1CB442F5D3CA
:10C190003046F8BD10B50446FCF708F8EE20FBF772
:10C1A000D8FFFCF73CF82046FBF7D3FFFCF737F845
:10C1B000FBF7FCFFEF20FBF7CCFFFCF730F800208B
:10C1C000FBF79AFF0446FCF70CF8204610BD7047B9
:10C1D00070B50D460446FBF7E9FFEE20FBF7B9FF0B
:10C1E000FCF71DF82046FBF7B4FFFCF718F82846CB
:10C1F000FBF7AFFFFCF713F8FBF7F3FF0A20FEF79E
:10C20000A6FA70BDF0B50025102605279C463F070D
:10C210000B46BE620C4C06E0595DE160A168C9079F
:10C22000FCD0E1686D1C8542F6DB002007E061462A
:10C23000095CE160A168C907FCD0E168401C90423C
:10C24000F5D3BE610020F0BD0030014000000102C6
:10C2500003040005405C0000A05C0400C06C080002
:10C26000805C0400E03F1E00E07D1E0007A902255F
:10C2700070889B880A001600010006000100020079
:10C2800087008D002D001A3152001A339A001A359A
:10C290001D011A376B003B31BE003B335E013B355D
:10C2A00096023B37000099599959EB518F421E4530
:10C2B000142E0080EB51F5283333E13A703DE13A1A
:10C2C000C235852BC2353333C235C235AE47E13A6C
:10C2D0005138A33051380000000000000000010276
:10C2E000030406070809030406080C101820300090
:10C2F0000000000102030400000000000000F03F05
:10C30000000000000000F83F0000000000000000F6
:10C310000000004003B8E23F000000000000000001
:10C3200006D0CF43EBFD4C3E033333333333E33F8F
:10C33000FFAB6FDBB66DDB3F4D268F515555D53FBB
:10C3400001411DA96074D13F65DBC9934A86CD3F89
:10C35000EF4E454A287ECA3F3E5555555555C53F77
:10C3600093BDBE166CC166BF2CDE25AF6A56113F69
:10C37000F16BD2C541BDBBBED0A4BE726937663E6B
:10C380000000000000000000A8C30008000000201A
:10C3900090010000BC5A00080CC400089001002065
:10C3A000681A0000ACA400080124130704380D0922
:10C3B0001E080540082609104008560A131D043BB4
:10C3C00008BE0516D8BC4010085201033AC84207FF
:10C3D0007052030CE5800C1B0202DD1409010222DD
:10C3E00081F01F6681049889968696798215980354
:10C3F0009814988796749778824397889671977760
:0CC400008249F10139293F92049220008A
:04000005080050C1DE
:00000001FF
